:100000000C9484090C94B9090C94B9090C94B9099D
:100010000C94B9090C94B9090C94B9090C94B90958
:100020000C94B9090C94B9090C94B9090C94A21A4E
:100030000C94B9090C94B9090C94B9090C94CC1618
:100040000C94B9090C94B9090C94B9090C94B90928
:100050000C9466430C9489430C94B9090C94B90927
:100060000C94B9090C94B9090C94B9090C94B90908
:100070000C94B9090C94B9090C94B9090C94B909F8
:100080000C94B9090C94B9090C94B909436C6561D5
:1000900072696E67205374617473000A696E7661C9
:1000A0006C696420646174650A005265706F7274D3
:1000B00020696E74657276616C3D25640A20456E18
:1000C000746572206E65773A20000A53657474690E
:1000D0006E67204D5050542062617420676F616CD0
:1000E0002025730A000A53657474696E67204D50A9
:1000F0005054204D6F64652025730A000A536574BF
:1001000074696E6720457870657274204D6F646500
:100110002025730A0025642D253032643A253032BB
:10012000643A25303264004C6F61642020252D38FC
:100130002E316620202020252D382E316620252DB9
:10014000382E316620202020252D382E316600499A
:100150006E20202020252D382E31662020202025BD
:100160002D382E316620252D382E31662020202076
:10017000252D382E31660020202020202043686164
:1001800072676528416829202050777228572920F6
:1001900020205065616B5077722857292020456ECA
:1001A0006572677928576829206F76657220252E39
:1001B00030662073656300252D362E326620252D8E
:1001C000342E32660A00252D362E326620252D3635
:1001D0002E326620252D362E326620252D362E32E3
:1001E00066252D362E326620252D342E32662025AA
:1001F0002D352E3166202564202564202564202598
:100200002D362E326620252D342E32660A000A53F2
:10021000657474696E67204C43442025730A006D31
:100220007070745F7363616E5F696E74657276611E
:100230006C3D2564206D696E0A20456E74657220E0
:100240006E65773A20004F4B0A000A536574746953
:100250006E672041545820534220506F77657220BA
:1002600025730A000A53657474696E6720415458F7
:1002700020506F7765722025730A0041545820532F
:1002800069672E205057525F4F4B2025730A00415B
:100290005458205369672E2050535F4F4E2020251D
:1002A000730A004154582050575220202020202506
:1002B000730A0041545820534220505752202025A1
:1002C000730A004368616E6765204F7363696C6CE5
:1002D00061746F722E204E6F77204F534343414C11
:1002E0003D25640A20456E746572206E65773A205C
:1002F0000020554252524C3D25642000204F53436C
:1003000043414C3D2564200020556E757365642083
:10031000737461636B203D25640020467573653AF4
:100320002065653D253032782068663D253032787D
:10033000206C663D25303278206C623D2530327865
:10034000004D43553D2530366C7800252D31306CFD
:100350007520252D31306C7520252D31306C7520A0
:10036000252D31306C7520252D31306C7520252DD3
:1003700031306C7520252D31306C750A00565F695F
:100380006E3E4D617820202056206261743E4D61A2
:100390007820204120696E3E4D6178202020412048
:1003A0006C6F61643E4D61782054206261743E4DF3
:1003B0006178202054206D69737320636E74204C23
:1003C000564420636E740A00446174652020202026
:1003D00020202054696D6520202020204261742057
:1003E000202020476F616C202020496E2020202093
:1003F00020615F696E202050574D20207077725F1A
:10040000696E20206D70707420207077722D646981
:1004100066660A0044617465202020202020205454
:10042000696D652020202020416828696E292020E0
:10043000204168286C6F61642920205028696E294A
:10044000202050286C6F61642920205128696E2972
:10045000202051286C6F6164290A00446174652072
:1004600020202020202054696D652020202020425B
:10047000617420202020476F616C202020496E206D
:1004800020202020615F696E202050574D2020548D
:100490005F426174207431202074322020765F6CBA
:1004A0006F616420615F6C6F61640A0043757272F2
:1004B000656E742064656275673D3078255820202C
:1004C0004E65773A2000445F504F5745523D307893
:1004D00025780A00445F4C45443D307825780A0071
:1004E000445F4F573D307825780A00445F4D5050A7
:1004F000545F5343414E5F424553543D3078257815
:100500000A00445F4D5050545F5343414E3D307894
:1005100025780A00445F4D5050543D307825780AC4
:1005200000445F4C4F41443D307825780A00445FD9
:100530004348415247453D307825780A00445F4F93
:100540005045523D307825780A00456E746572201A
:100550004F6E2D426F6172642074656D70207365FB
:100560006E736F72206964783A2000456E7465720C
:1005700020426174746572792074656D70207365B2
:100580006E736F72206964783A20004261747465FA
:1005900072792054656D70203D2025352E3266001D
:1005A000765F6C76645F687973743D25352E3266AC
:1005B0000A20456E746572206E65773A2000765F7A
:1005C0006C76643D25352E32660A20456E74657260
:1005D000206E65773A20004C6F61642063757272FB
:1005E000656E74206C696D69743D25352E32660A1E
:1005F00020456E746572206E65773A2000496E70F2
:1006000075742063757272656E74206C696D69749F
:100610003D25352E32660A20456E746572206E6562
:10062000773A2000765F676F616C5F6C6F61643D45
:1006300025352E32660A20456E746572206E657708
:100640003A2000765F676F616C3D25352E32660A71
:1006500020456E746572206E65773A2000666C7472
:100660005F666163746F723D25352E32660A2045E0
:100670006E746572206E65773A2000666C74206631
:100680006163746F7220636F6E74726F6C73207429
:10069000686520706572696F64206265666F726557
:1006A000206E65787420626F6F7374207065726954
:1006B0006F640A00506C65617365207365742079FE
:1006C0006F757220666978656420766F6C746167F7
:1006D0006525730A000A53657474696E672046695C
:1006E00078656420566F6C74616765204D6F646532
:1006F0002025730A006174787320202D207365749F
:100700002041545820534220706F77657220257322
:100710000A006174787020202D2041545820706F99
:100720007765722025730A00726920202D2072657A
:10073000706F727420696E74657276616C20696E78
:10074000207365630A0D00727320202D207265737B
:10075000746F72652064656661756C74207365746E
:1007600074696E67730A0D006F7720202D206F77F4
:100770002D6275732064756D700A0D006D692020FF
:100780002D20736574204D505054207363616E208A
:10079000696E74657276616C0A006D6220202D208E
:1007A000736574204D505054206261747465727981
:1007B0002025730A006D7420202D20736574204D50
:1007C0005050542025730A006C7020202D20736532
:1007D00074204C43442025730A00646920202D2096
:1007E000646973636F6E6E65637420696E7075748F
:1007F000206D616E75616C6C790A0D006369202053
:100800002D20636F6E6E65637420696E7075742041
:100810006D616E75616C6C790A0D00646C20202D21
:1008200020646973636F6E6E656374206C6F6164BE
:10083000206D616E75616C6C790A0D00636C20200F
:100840002D20636F6E6E656374206C6F6164206D24
:10085000616E75616C6C790A0D00762020202D2068
:1008600076657273696F6E0A0D00752020202D2049
:10087000757074696D650A0D00747320202D2074E5
:10088000696D65207365740A0D00636320202D2057
:1008900063686172676520737461747320636C654B
:1008A00061720A0D00637320202D206368617267F6
:1008B000652073746174730A0D00742020202D204C
:1008C00074696D652073686F770A0D006465202078
:1008D0002D2064656275670A0D00737320202D203A
:1008E0007374617475732073756D6D6172790A0D1F
:1008F00000626D20202D206261747465727920730E
:1009000075626D656E750A0D00682020202D2068C7
:10091000656C700A0D00756E6B6E6F776E20636D7F
:10092000640A006D2020202D206261636B20746FAB
:10093000206D61696E206D656E750A0D007268200C
:10094000202D207265636F6E6E6563742068797305
:100950007465726573697320766F6C746167650A7C
:100960000D00647620202D20646973636F6E6E65C0
:10097000637420766F6C746167650A0D00766C2075
:10098000202D20766F6C74616765206C6F61642028
:10099000676F616C0A0D00666620202D20666C6F03
:1009A000617420706572696F6420666163746F7230
:1009B0000A0D00766720202D20766F6C74616765C4
:1009C00020676F616C0A0D00667620202D20626121
:1009D000747465727920666978656420766F6C74CA
:1009E000616765206D6F64650A0D00626120202DCE
:1009F000206261747465727920766F6C74616765CA
:100A000020706172616D730A0D00746920202D20C1
:100A1000626174746572792073656E736F72206F92
:100A20006E652D7769726520696E6465780A0D00C0
:100A3000746520202D20626174746572792074655C
:100A40006D70657261747572650A0D0063612020B6
:100A50002D2063616C69627261746520766F6C74BD
:100A60006167652072656164696E67730A0D006174
:100A70006C20202D206C696D6974206C6F6164207E
:100A800063757272656E740A0D00616920202D20F5
:100A90006C696D697420696E70757420637572720B
:100AA000656E740A0D00646520202D2064656275F2
:100AB000670A0D00682020202D2068656C700A0DE3
:100AC00000426F6F737420566F6C746167652061AC
:100AD0007420323043203D25352E32660A20456E83
:100AE000746572204E65773A2000466C6F61742001
:100AF000566F6C7461676520617420323043203D0D
:100B000025352E32660A20456E746572204E657753
:100B10003A2000496E2043757272656E743D25352A
:100B20002E32660A20456E74657220636F7272659C
:100B3000637465643A20004C6F616420437572727F
:100B4000656E743D25352E32660A20456E746572D9
:100B500020636F727265637465643A20004C6F6144
:100B60006420566F6C746167653D25352E32660AC8
:100B700020456E74657220636F727265637465647C
:100B80003A2000496E70757420566F6C7461676509
:100B90003D25352E32660A20456E74657220636FDE
:100BA000727265637465643A2000426174746572A0
:100BB0007920566F6C746167653D25352E32660A63
:100BC00020456E74657220636F727265637465642C
:100BD0003A20005265706F727420696E7465727687
:100BE000616C203D25356420730A004C6F616420E0
:100BF000617665726167652063757272656E7420D7
:100C00003D25352E336620410A004C6F6164207605
:100C10006F6C7461676520676F616C203D25352EB0
:100C20003166560A004D505054207363616E20693E
:100C30006E74657276616C203D2564206D696E0A64
:100C4000004D505054207363616E3A2050574D2030
:100C500075736564203D2025642C206265737420C3
:100C60003D25642C205057523D25352E33660A0011
:100C70004D50505420765F626174203D25640A0017
:100C80004D505054206C6F636B2F6E6F6C6F636BA5
:100C9000203D256C752F256C750A0054656D7020FC
:100CA00062617474657279203D25362E3266204368
:100CB000202844656661756C74290A0054656D705E
:100CC0002073656E736F72206572726F72203D259E
:100CD0006420430A00202844656661756C742920ED
:100CE0005741524E494E472074656D702073656EB2
:100CF000736F72206964206E6F7420636F6E666913
:100D000067757265640054656D7020626174746506
:100D10007279203D25362E3266204300566F6C7462
:100D2000616765206C6F6164207265636F6E6E65CC
:100D30006374206F6666736574203D25352E3266B8
:100D400020560A00496E707574206973206D616EBB
:100D500075616C6C7920646973636F6E6E65637422
:100D600065640A004C6F6164206C6173742064696F
:100D700073636F6E6E656374656420004C6F6164AD
:100D8000206973206D616E75616C6C792064697384
:100D9000636F6E6E65637465640A004C6F616420F6
:100DA0006973206C6F7720766F6C7461676520645F
:100DB0006973636F6E6E65637465640A00566F6C69
:100DC00074616765206C6F616420646973636F6E22
:100DD0006E656374203D25352E316620560A004C21
:100DE0006173742063686172676520004D617820CB
:100DF0006C6F61642063757272656E74203D253579
:100E00002E316620410A004D617820696E7075743C
:100E10002063757272656E74203D25352E31662013
:100E2000410A0043757272656E74206C6F616420B4
:100E30003D25362E336620410A0043757272656E79
:100E40007420696E203D25362E336620410A0056F7
:100E50006F6C74616765206C6F6164203D25352E71
:100E6000326620560A00566F6C7461676520676FA2
:100E7000616C203D25352E3166560A00566F6C7424
:100E800061676520666C6F6174203D25352E316683
:100E9000560A00566F6C7461676520626F6F7374D9
:100EA000203D25352E3166560A00566F6C746167F9
:100EB0006520696E203D25352E326620560A005683
:100EC0006F6C7461676520626174203D25352E3238
:100ED0006620560A00566F6C746167652063617006
:100EE000203D25352E326620560A004C564420748B
:100EF000696D652000557074696D652000446174EA
:100F0000652000312E300D0A0020257320537461B6
:100F1000727420005254432025732C00436F707963
:100F20007269676874204865726A756C66205574CA
:100F30007665636B6C696E672C2055707073616C9D
:100F4000612053776564656E2C206865726A756CE4
:100F5000662E73650D0A004669726D7761726520B1
:100F60005665722E20362E3420323031332D3130FA
:100F70002D30340D0A0020252D382E316620252DE8
:100F8000382E316620252D382E316620252D382E1D
:100F9000316620252D382E306620252D382E3066DE
:100FA0000A004368617267652074696D6572206527
:100FB0007870697265642061667465722025752099
:100FC0007365630A00426F6F7374207265616368B2
:100FD000656420696E2025752073656320666C74D6
:100FE0002D706572696F642073657420746F20259D
:100FF00075207365630A00204D505054207363615F
:101000006E20646F6E653A2050574D20757365648D
:10101000203D202534642C2062657374203D2534E6
:10102000642C205057523D25352E33660A00204D42
:10103000505054207363616E3A2050574D207573A1
:101040006564203D202534642C207363616E203D4F
:101050002534642C205057523D25352E33660A0026
:1010600020252D362E326620252D362E326620255F
:101070002D362E326620252D342E326620253464FE
:101080002020252D372E33662025642020252D375E
:101090002E3366200A0020252D362E326620252D7F
:1010A000362E326620252D342E3266202534640AF1
:1010B0000020252D362E326620252D362E32662034
:1010C000252D362E326620252D342E3266202534ED
:1010D0006420252D352E31662025642025642025A9
:1010E0006420252D362E326620252D342E32660AB8
:1010F00000253034642D253032642D2530326420B3
:10110000253032643A253032643A25303264007436
:101110005F626174203D2025362E32660A005761D9
:10112000726E696E672E20426174746572792073E5
:10113000656E736F72206964206E6F7420736574BE
:101140000A005761726E696E672E204E6F207465BB
:101150006D702073656E736F72730A0052657365EC
:101160007474696E6700526573746F726520616C88
:101170006C2073657474696E67733F20792F6E3AC3
:101180002000253034642D253032642D2530326422
:1011900020253032643A253032643A2530326400FA
:1011A00020257300204F6E2D426F61726400204233
:1011B000617474657279002025362E326620002510
:1011C00030327800256420000A006E616E00696E7E
:1011D000660000407A10F35A00A0724E1809001001
:1011E000A5D4E80000E87648170000E40B5402009C
:1011F00000CA9A3B000000E1F505000080969800C7
:10120000000040420F000000A086010000001027EF
:1012100000000000E803000000006400000000007F
:101220000A00000000000100000000002C76D888B1
:10123000DC674F0823DFC1DFAE59E1B1B796E5E3C4
:10124000E453C63AE651997696E8E6C28426EB89DD
:101250008C9B62ED407C6FFCEFBC9C9F40F2BAA57A
:101260006FA5F490055A2AF75C936B6CF9676DC112
:101270001BFCE0E40D47FEF520E6B500D0ED902E16
:101280000300943577050080841E080000204E0A74
:10129000000000C80C333333330F986E12831141B2
:1012A000EF8D2114893BE65516CFFEE6DB18D1847D
:1012B0004B381BF77C1D901DA4BBE42420328472A4
:1012C0005E228100C9F124ECA1E53D27494E464943
:1012D0004E4954594E414ECDCCCC3D0AD7233C17F4
:1012E000B7D13877CC2B329595E6241FB14F0A0041
:1012F0000020410000C84200401C4620BCBE4CCA31
:101300001B0E5AAEC59D7400EDEBF3E085EC90E446
:1013100001C08193EF3FF907E0F3D9F311241FBE19
:10132000CFEFD0E4DEBFCDBF84B78093BC0314BE43
:1013300088E10FB6F89480936000109260000FBEB1
:1013400011E0A0E0B1E0E2EEF5EA00E00BBF02C080
:1013500007900D92A23CB107D9F713E0A2ECB1E0DF
:1013600001C01D92AC3BB107E1F70E94C9380C9453
:10137000EF520C940000209170002C7F209370009D
:101380000097C1F081E08093A6018091B600806251
:101390008093B6001092B20082E08093B1008091F9
:1013A000B60090E0877090700097C9F781E0809355
:1013B000700008951092A6011092B2008091B600BC
:1013C0008F7D8093B60086E08093B1008091B60057
:1013D00090E0877090700097C9F781E0809370006B
:1013E0000895AF92BF92CF92DF92EF92FF920F9348
:1013F0001F93CF93DF937B018C018DB79EB70A9724
:101400000FB6F8949EBF0FBE8DBFCDB7DEB7219645
:1014100085E191E0EDB7FEB792838183C801B70102
:1014200020E831E541E050E00E94AB4B3B832A834A
:1014300030E1A32E3EE0B32EC12CD12CA6019501A4
:101440000E94AB4B332727FD30953D832C83C80189
:10145000B701A60195010E94AB4B2CE3A22EB12C43
:10146000C12CD12CA60195010E94AB4B332727FD3F
:1014700030953F832E83C801B701A60195010E94D4
:10148000AB4B772767FD7095798768870E94EB4E95
:101490008DB79EB708960FB6F8949EBF0FBE8DBF4E
:1014A00088EC91E1EDB7FEB7928381830E94EB4E09
:1014B0000F900F90DF91CF911F910F91FF90EF90C0
:1014C000DF90CF90BF90AF900895EDEBF3E080E414
:1014D000EF3FF80709F0A8F420E030E005C080E411
:1014E000EF3FF80709F058F431968081853CB9F751
:1014F0002F5F3F4F80E4EF3FF807B1F3A8F3C90136
:10150000089520E030E0FBCF009749F410924601A7
:101510001092C2010A9A1298089A1098089581E0D0
:10152000809346010898109A0895009739F40A9A12
:1015300012981092C201229A2A98089522982A9A03
:1015400008956F927F928F929F92AF92BF92CF92A7
:10155000DF92EF92FF920F931F93DF93CF93CDB75C
:10156000DEB729970FB6F894DEBF0FBECDBF10923D
:10157000D7018FEF89837FE3C72E72E0D72EEE2449
:10158000FF24882462E0A62EB12CAC0EBD1E3E01C5
:101590000894611C711C8E01065F1F4F9E2CC301B5
:1015A000B5010E94774189818F3F09F485C08E3F44
:1015B00009F482C0C5010E949241F6018087F501BD
:1015C000D701AA0FBB1FAA0FBB1FAA0FBB1FAE0DCF
:1015D000BF1DA15CBD4F81918D93E017F107D9F735
:1015E0009091BB02F60180819817D1F19394898183
:1015F000882369F00894E11CF11C89E090E0C80E92
:10160000D91E98E0E916F10449F648E0942E8820A6
:1016100089F48FEF8093BB028093BC028093BD025C
:101620008093BE028093BF028093C0028093C10268
:101630008093C202892D29960FB6F894DEBF0FBEA3
:10164000CDBFCF91DF911F910F91FF90EF90DF9071
:10165000CF90BF90AF909F908F907F906F900895A4
:101660009091BC028181981709F69091BD02828108
:10167000981709F0BBCF9091BE028381981709F0AB
:10168000B5CF9091BF028481981709F0AFCF9091A8
:10169000C0028581981709F0A9CF9091C102868177
:1016A000981709F0A3CF9091C2028781981709F08B
:1016B0009DCF882483949ACF8093D701A8CF0E948E
:1016C000A10A8093D601089500D088EC91E1EDB78E
:1016D000FEB7928381830E94EB4E0F900F90089586
:1016E0002F923F924F925F926F927F928F929F9232
:1016F000AF92BF92CF92DF92EF92FF920F931F9320
:10170000CF93DF930E945F0B8091D601882309F469
:10171000BEC0CFE3D2E0AA24BB24B4EC4B2EB1E18F
:101720005B2EAFEBCA2EA1E1DA2EF7EB2F2EF1E103
:101730003F2E00D000D0ADB7BEB712965C924E924D
:1017400011971496BC92AE9213970E94EB4E0F9095
:101750000F900F900F908501000F111F000F111FA8
:10176000000F111F0A0D1B1D015C1D4FC8010E94B7
:10177000D742FC01BF01882777FD8095982F0E94F2
:10178000614A3B014C01780100E010E0D7018D91E6
:101790007D0100D000D0EDB7FEB73196ADB7BEB732
:1017A0001296DC92CE921197828313820E94EB4EA6
:1017B0000F5F1F4F0F900F900F900F900830110583
:1017C00029F700D000D000D00DB71EB70F5F1F4F14
:1017D000EDB7FEB732822182662D772D882D992DA7
:1017E00020E030E048EC52E40E94C649D80112964D
:1017F0006D937D938D939C9315970E94EB4E8881FA
:1018000029813A81EB817C816D815E814F81ADB709
:10181000BEB716960FB6F894BEBF0FBEADBF90917F
:10182000BB02981709F47AC090911703981709F42E
:1018300044C088858823F1F180E091E000D000D099
:10184000E0EAF1E1ADB7BEB71296FC93EE931197C3
:1018500014969C938E9313970E94EB4E0F900F90CB
:10186000E8ECF1E1ADB7BEB71296FC93EE93119799
:101870000E94EB4E0894A11CB11C29968091D601C0
:1018800090E00F900F90A816B9060CF452CFDF919C
:10189000CF911F910F91FF90EF90DF90CF90BF906D
:1018A000AF909F908F907F906F905F904F903F9000
:1018B0002F90089589E091E0C1CF8091180382179D
:1018C00009F0B7CF80911903831709F0B2CF809147
:1018D0001A038E1709F0ADCF80911B03871709F00B
:1018E000A8CF80911C03861709F0A3CF80911D0318
:1018F000851709F09ECF80911E03841709F099CFB8
:1019000000D0E4EAF1E1ADB7BEB71296FC93EE93D6
:1019100011970E94EB4E0F900F908BCF9091BC02CD
:10192000921709F081CF9091BD02931709F07CCFF7
:101930009091BE029E1709F077CF9091BF02971742
:1019400009F072CF9091C002961709F06DCF909177
:10195000C102951709F068CF9091C202941709F05F
:1019600063CF00D02EEA31E1EDB7FEB73283218399
:101970000E94EB4E888129813A81EB817C816D81C7
:101980005E814F810F900F904FCFEAE7F0E080E843
:10199000808380818760808310927B0088EF8093B2
:1019A0007E00808188608083808180648083089548
:1019B00080937C0080917C00806C80937C0086E02A
:1019C00080937A0080917A00806880937A00809179
:1019D0007A00806480937A0080917A0086FDFCCF43
:1019E00088E090E060E070E020917A00206420932D
:1019F0007A0020917A0026FDFCCF2091780030916A
:101A00007900620F731F019779F780917A008F77C1
:101A100080937A0076956795769567957695679524
:101A200080E090E00E945F4A0895CF92DF92EF92AB
:101A3000FF920F931F93CF93DF937B018C016A0179
:101A4000E901FA018081882371F4C801B70120E01F
:101A500030E0A9010E94114B18160CF054C0649795
:101A6000109201020CC0C801B70120E030E0A901CA
:101A70000E94114B181604F5649610920102809191
:101A8000EC019091ED01A091EE01B091EF01019672
:101A9000A11DB11D8093EC019093ED01A093EE0187
:101AA000B093EF01CE01DF91CF911F910F91FF9085
:101AB000EF90DF90CF900895C801B70120E030E0AB
:101AC000A9010E94C24987FD31C0809101028F5F48
:101AD00080930102823098F28150809301028091BC
:101AE000E8019091E901A091EA01B091EB01019622
:101AF000A11DB11D8093E8019093E901A093EA0133
:101B0000B093EB01CFCFC801B70120E030E0A901CD
:101B10000E94C24987FFD9CF81E0F6018083649695
:101B2000809101028F5F80930102D4CF6497F60108
:101B30001082809101028F5F80930102CBCFEF92E0
:101B4000FF920F931F93CF93DF93609113037091D4
:101B5000140380911503909116032091FF02309198
:101B6000000340910103509102030E94114B18168B
:101B70000CF580919A0190919B0123E08F3F920791
:101B800028F580919A0190919B01E0919C01F09140
:101B90009D01909399018093980180919801909173
:101BA000990191838083DF91CF911F910F91FF90D5
:101BB000EF9008958091DE01882359F080919A0179
:101BC00090919B0133E08F3F9307D8F28FEF93E022
:101BD000DCCF60910F0370911003809111039091FD
:101BE0001203E0907101F090720100917301109165
:101BF0007401A80197010E94114B18160CF063C0E4
:101C000060910F0370911003809111039091120362
:101C1000A80197010E945D4920E030E0A9010E94DF
:101C2000114B18160CF057C060910F037091100300
:101C30008091110390911203A80197010E945D49C0
:101C400020E030E048E452E40E94154B0E94334A01
:101C50008091980190919901860F971F97FDF6C08A
:101C600020919A0130919B012817390720F4809127
:101C70009A0190919B01E0919C01F0919D019093BC
:101C80009901809398018091980190919901918395
:101C900080838091A3029091A402A091A502B091AB
:101CA000A6020196A11DB11D8093A3029093A402E8
:101CB000A093A502B093A602DF91CF911F910F913F
:101CC000FF90EF900895809100021816D4F481508F
:101CD0008093000268CF60910F0370911003809190
:101CE000110390911203A80197010E945D49905839
:101CF00020E030E048E452E40E94154B0E94334A51
:101D0000A7CF8091FE019091FF0101969093FF0172
:101D10008093FE0180918F0290919002A091910298
:101D2000B091920280930B0390930C03A0930D0348
:101D3000B0930E0380918B01882309F4A6C06091B3
:101D40001303709114038091150390911603209151
:101D50000F033091100340911103509112030E9420
:101D6000154B9B01AC0120938F023093900240935E
:101D70009102509392026091610170916201809191
:101D800063019091640120911303309114034091F9
:101D90001503509116030E945D4920E030E0A9012F
:101DA0000E94114B18160CF054C0609161017091A3
:101DB000620180916301909164012091130330913D
:101DC000140340911503509116030E945D4920E0D1
:101DD00030E048E452E40E94154B0E94334AE62E5C
:101DE000E7017E01F72EE701CF31D10510F0CEE1FA
:101DF000D0E06091FF027091000380910103909107
:101E00000203E0901303F090140300911503109166
:101E100016032DEC3CEC4CE45EE30E945D49A80106
:101E200097010E94114B1816CCF180919801909166
:101E300099018C0F9D1F97FDFFC020919A01309151
:101E40009B012817390708F49CCE9FCE80E090E0D4
:101E500012CF609161017091620180916301909154
:101E600064012091130330911403409115035091A4
:101E700016030E945D49905820E030E048E452E4A7
:101E80000E94154B0E94334AAACF6091FF027091C5
:101E90000003809101039091020359CF60911303D5
:101EA00070911403809115039091160320916101A4
:101EB0003091620140916301509164010E94114B85
:101EC00018169CF580919801909199018C0F9D1F97
:101ED00097FDB5C020919A0130919B0128173907D1
:101EE00020F480919A0190919B01E0919C01F091E6
:101EF0009D01909399018093980180919801909110
:101F00009901918380836091B7027091B8028091AA
:101F1000B9029091BA0220E030E0A9010E94C249C2
:101F200087FF41CE1092D1013ECE60911303709194
:101F30001403809115039091160320916101309153
:101F4000620140916301509164010E94C24987FF80
:101F50002ACE80918A01882309F466C08091D1013C
:101F6000882309F4DFC060918F0270919002809104
:101F70009102909192022091B7023091B802409163
:101F8000B9025091BA020E94114B18160CF4B1C05C
:101F90002091FC013091FD012115310509F052C05D
:101FA000809198019091990190933E0280933D0217
:101FB00084E690E03093C7022093C6029093FD011F
:101FC0008093FC0120919A0130919B0128173907D9
:101FD00020F480919A0190919B01E0919C01F091F5
:101FE0009D0190939901809398018091980190911F
:101FF00099019183808380918F0290919002A091AA
:102000009102B09192028093210390932203A093B6
:102010002303B093240380912003886080932003DE
:1020200087E080930002BFCD809198019091990143
:102030008C1B9D0B97FF01CF80E090E0A6CD80E048
:1020400090E053CFC9018C599F4F43E08F3F9407D5
:1020500008F4B0CF1092D1018091C4029091C502D2
:1020600097FDB7C020919A0130919B01281739073D
:1020700020F480919A0190919B01E0919C01F09154
:102080009D0190939901809398018091980190917E
:102090009901918380838091B7029091B802A091B9
:1020A000B902B091BA028093210390932203A093C6
:1020B0002303B093240380E090E0A0E8BFEB80937B
:1020C000B7029093B802A093B902B093BA0280917C
:1020D000C4029091C5029093C7028093C6021092E9
:1020E000FD011092FC018091200380618093200308
:1020F00097CF2091FC013091FD013093C5022093D0
:10210000C40280918F0290919002A0919102B091AF
:1021100092028093B7029093B802A093B902B09351
:10212000BA023ACF85E08093000260918F027091ED
:102130009002809191029091920220910B03309134
:102140000C0340910D0350910E03C0919801D09162
:1021500099010E945D494BEA51E09E010E94150DD4
:1021600090939901809398018091980190919901A1
:1021700023E08F3F920734F16091130370911403B1
:102180008091150390911603E0906101F090620137
:1021900000916301109164012DEC3CEC4CE45EE392
:1021A0000E945E49A80197010E94C24987FF14C09E
:1021B0008091C4029091C5029093990180939801F7
:1021C0001092AB01809198019091990197FD34CFC5
:1021D00034CE80E090E051CF8FEF93E0909399015F
:1021E00080939801EFCFCF92DF92EF92FF920F93FF
:1021F0001F93CF93DF93609193027091940280912B
:10220000950290919602209175013091760140914E
:102210007701509178010E94114B1816ECF58091CE
:102220008C0190918D0184539F4F97FDBDC02091EB
:102230008E0130918F012817390720F480918E018B
:1022400090918F01E0919001F091910190938D0117
:1022500080938C0180918C0190918D01918380837A
:102260008091A7029091A802A091A902B091AA0220
:102270000196A11DB11D8093A7029093A802A0937F
:10228000A902B093AA02DF91CF911F910F91FF9005
:10229000EF90DF90CF9008958091DD018823E1F0E9
:1022A00080918E0190918F0123E08F3F920708F07B
:1022B0007EC080918E0190918F01E0919001F0910C
:1022C000910190938D0180938C0180918C0190916C
:1022D0008D0191838083D7CF8091DC01882301F722
:1022E000E0906501F090660100916701109168012E
:1022F00020913102309132024091330250913402E8
:10230000C801B7010E945D4920E030E0A9010E94A8
:10231000114B18160CF068C0209131023091320236
:102320004091330250913402C801B7010E945D49C7
:1023300020E030E048E452E40E94154B0E94334A0A
:10234000C62EE6016E01D72EE601C430D10510F08D
:10235000C3E0D0E02091310230913202409133024B
:1023600050913402C801B7010E94C24987FF22C0C0
:1023700080918C0190918D018C0F9D1F33E08D3FDA
:10238000930708F047C080918C0190918D018C0FCC
:102390009D1F97FD26C020918E0130918F01281737
:1023A000390708F486CF89CF80E090E04BCF8FEFDC
:1023B00093E083CF20913102309132024091330279
:1023C00050913402C801B7010E94114B18160CF04D
:1023D0005ACF80918C0190918D018C1B9D0B97FFA2
:1023E000DACF80E090E069CF209131023091320263
:1023F0004091330250913402C801B7010E945D49F7
:10240000905820E030E048E452E40E94154B0E94CE
:10241000334A96CF80918C0190918D01CCEFD3E01F
:10242000C81BD90BB0CF94B1936094B995B19360A8
:1024300095B9833081F0843038F0863091F0873060
:1024400039F0853041F00895813021F0823028F054
:102450002998089529982898089585B1836085B9A9
:102460000895299885B1817085B90895CF93DF9338
:102470008FE192E020911F0230912002FC01319700
:10248000A081FC0132977081FC0133976081FC01CF
:10249000349750810597EC014881EDB7FEB73E9720
:1024A0000FB6F894FEBF0FBEEDBF319682E891E102
:1024B000CDB7DEB79A83898333832283A4831582C1
:1024C0007683178260871186528713864487158624
:1024D0000E94EB4EEDB7FEB73E960FB6F894FEBFE6
:1024E0000FBEEDBFDF91CF910895AAE1B2E0E9EA16
:1024F000F3E087E001900D928150E1F70895CF93CA
:10250000DF93ECE9F1E0A0919C01B0919D01EF0116
:1025100022978881998134979183808380819181EA
:1025200011969C938E935D98DF91CF910895E0E88A
:10253000F0E020EC20832081236020832AE0209398
:102540008100A8E8B0E011969C938E938D919C91A8
:102550001197559A8081806380838FEF91E09093EB
:102560008D0180938C0190938B0080938A00549A04
:1025700081E080936F008FEF93E090938F018093C1
:102580008E0190939B0180939A01789408958FEF28
:1025900081B911B812B884B914B815B887B917B889
:1025A00018B88AB91AB81BB80F980E980D980C98DD
:1025B0000B9888EF80937E00399A419A389A409A16
:1025C000579A5F9A8091C40181FF0BC080914701A7
:1025D000882309F4D2C081E090E00E94950A80919E
:1025E000C40180FF09C080914601882309F0CCC056
:1025F00080E090E00E94840A81E090E00E94BB09A4
:1026000081E791E06DE270E044E050E00E94A04F6D
:1026100085E791E061E370E044E050E00E94A04F64
:1026200089E791E066E370E044E050E00E94A04F4B
:1026300081E691E06DE170E044E050E00E94A04F3F
:1026400085E691E061E270E044E050E00E94A04F36
:1026500089ED91E065E370E041E050E00E94A04F19
:102660008BEB92E066E470E049E050E00E94A04FFE
:1026700087E193E06FE470E049E050E00E94A04FF2
:1026800088E591E06CE070E044E050E00E94A04FEB
:102690008CE591E060E170E044E050E00E94A04FE2
:1026A00085EC91E064E170E044E050E00E94A04FCE
:1026B00089EC91E068E170E044E050E00E94A04FB6
:1026C00080E591E064E070E044E050E00E94A04FBB
:1026D00084E591E068E070E044E050E00E94A04FA3
:1026E0008CE491E060E070E044E050E00E94A04F94
:1026F0008DE791E06AE370E044E050E00E94A04F73
:1027000089E691E065E270E044E050E00E94A04F6D
:102710008DE691E069E270E044E050E00E94A04F55
:1027200082E891E06EE370E044E050E00E94A04F48
:102730008AE891E062E470E044E050E00E94A04F3B
:102740008BE891E063E470E044E050E00E94A04F29
:1027500080E691E06CE170E041E050E00E94A04F23
:1027600085EE91E064E470E042E050E00E94A04F0A
:102770008FEF93E00E949712089580E090E00E940E
:10278000950A8091C4012DCF81E090E00E94840AD7
:1027900033CFEF92FF920F931F93CF93DF938091EC
:1027A000D601882309F4ADC08091BB028F3F09F4A4
:1027B00056C08BEB92E00E94D7429C01B90188275A
:1027C00077FD8095982F0E94614A20E030E048EC28
:1027D00052E40E94C649E62EF72E082F192F2091A9
:1027E000D2013091D30126FDB7C0C801B70120E066
:1027F00030E048EA52E40E94114B1816FCF41092A3
:10280000D6018091AB029091AC02A091AD02B09143
:10281000AE020196A11DB11D8093AB029093AC0254
:10282000A093AD02B093AE020F2EF0E0EF2EF0E0D9
:10283000FF2EF8EC0F2FF1E41F2FF02DF894E0920B
:102840004801F092490100934A0110934B0178949A
:10285000DF91CF911F910F91FF90EF90089580919C
:10286000BC028F3F09F0A5CF8091BD028F3F09F0D8
:10287000A0CF8091BE028F3F09F09BCF8091BF0215
:102880008F3F09F096CF8091C0028F3F09F091CF22
:102890008091C1028F3F09F08CCF8091C2028F3F9F
:1028A00009F087CF8091AB029091AC02A091AD026C
:1028B000B091AE020196A11DB11D8093AB02909321
:1028C000AC02A093AD02B093AE028091D201909180
:1028D000D30186FF36C000D08EE191E1EDB7FEB79F
:1028E000928381830E94EB4E0F900F900F2EF0E0A9
:1028F000EF2EF0E0FF2EF8EC0F2FF1E41F2FF02D5C
:102900009DCF0E945F0B8091D601882309F04CCFA8
:102910008091AB029091AC02A091AD02B091AE0259
:102920000196A11DB11D8093AB029093AC02A093C0
:10293000AD02B093AE028091D2019091D30186FD99
:102940002AC00F2EF0E0EF2EF0E0FF2EF8EC0F2F54
:10295000F1E41F2FF02D72CF00D000D000D02FE077
:1029600031E1CDB7DEB73A832983262F372F482FA1
:10297000592FEDB7FEB723833483458356830E94D6
:10298000EB4E2DB73EB72A5F3F4F0FB6F8943EBFD0
:102990000FBE2DBF2ACF00D082E491E1CDB7DEB7C4
:1029A0009A8389830E94EB4E0F900F900F2EF0E0D8
:1029B000EF2EF0E0FF2EF8EC0F2FF1E41F2FF02D9B
:1029C0003DCF6091DF017091E0016115710551F417
:1029D00081E090E09093E0018093DF0168E873E18B
:1029E000CB01089588E893E10E94844B611571053D
:1029F000B9F761E070E0CB010895CF93DF93C09108
:102A0000DF01D091E0012097E9F0BE0180E090E085
:102A10000E945F4A9B01AC01609182017091830129
:102A200080918401909185010E94C6490E94334A99
:102A3000262F372F2C173D0708F49E01C901DF917F
:102A4000CF91089581E090E09093E0018093DF01C1
:102A500020E030E040E85FE3C1E0D0E0DDCF2F923E
:102A60003F924F925F926F927F928F929F92AF921E
:102A7000BF92CF92DF92EF92FF920F931F93DF935B
:102A8000CF9300D000D0CDB7DEB73B014C012091F1
:102A900048013091490140914A0150914B0160E059
:102AA00070E080EA91E40E945D4926EA3BE944EC4B
:102AB0005CE30E94154B20916D0130916E014091B5
:102AC0006F01509170010E945E49F62E072F182F5A
:102AD000E92E862F902FA12FBE2D89839A83AB8359
:102AE000BC83209148013091490140914A015091A5
:102AF0004B0160E070E080EA91E40E945D4926EAC3
:102B00003BE944EC5CE30E94154B20916901309154
:102B10006A0140916B0150916C010E945E495B011A
:102B20006C0115012601C401B3012F2D302F412F57
:102B30005E2D0E94114B87FD07C08091FA01909194
:102B4000FB01009709F49DC0809186019091870157
:102B5000009709F05CC0809120038064809320037B
:102B60008091DF019091E0019093E2018093E10177
:102B70008091FA019091FB018130910559F080918B
:102B8000F6019091F70101969093F7018093F60179
:102B900080FD63C020926101309262014092630126
:102BA00050926401609161017091620180916301B2
:102BB000909164012091FF02309100034091010344
:102BC000509102030E94114B1816C4F58CE390E05B
:102BD00090938701809386018091F8019091F9018B
:102BE000009709F447C0209261013092620140923F
:102BF0006301509264011092F9011092F801109251
:102C0000E0011092DF011092FB011092FA010F9087
:102C10000F900F900F90CF91DF911F910F91FF9028
:102C2000EF90DF90CF90BF90AF909F908F907F906C
:102C30006F905F904F903F902F90089588E790E0BD
:102C400090938701809386011092E0011092DF013A
:102C50001092FB011092FA01DACF89819A81AB813F
:102C6000BC818093610190936201A0936301B09352
:102C7000640198CF81E090E09093F9018093F8018E
:102C8000E3CFA0926101B0926201C0926301D09241
:102C900064010E94FD1490938701809386019093B4
:102CA000E4018093E3018091DF019091E001909332
:102CB000E2018093E10180912003806280932003F0
:102CC0001092E0011092DF0181E090E09093FB010F
:102CD0008093FA019CCFAF92BF92CF92DF92EF9296
:102CE000FF920F931F938091DA019091DB0100977F
:102CF00021F5609113037091140380911503909155
:102D00001603E0907901F0907A0100917B01109117
:102D10007C01A80197010E94C24987FF17C08091DA
:102D2000DC01882399F180918101882331F488E7BF
:102D300090E09093DB018093DA011F910F91FF9057
:102D4000EF90DF90CF90BF90AF900895A0901303C5
:102D5000B0901403C0901503D0901603C801B701BA
:102D600020917D0130917E0140917F015091800141
:102D70000E945E49A60195010E94C24987FFDDCFEE
:102D80001092DC018AE080938101D7CF809181018C
:102D9000815080938101C9CF1F920F920FB60F927D
:102DA0000BB60F921124EF92FF920F931F932F9364
:102DB0003F934F935F936F937F938F939F93AF93C3
:102DC000BF93EF93FF938091A9019091AA0101977E
:102DD0009093AA018093A901009709F001C1609125
:102DE000FF027091000380910103909102032091F2
:102DF00013033091140340911503509116030E9460
:102E0000114B18160CF403C110E0409887E00E94A3
:102E1000D80C2091500130915101409152015091B4
:102E200053010E94154B9B01AC0120931303309377
:102E3000140340931503509316036091130370918C
:102E40001403809115039091160320E030E048EDC3
:102E500051E40E94114B18169CF480919F029091AE
:102E6000A002A091A102B091A2020196A11DB11DE4
:102E700080939F029093A002A093A102B093A2021C
:102E800086E00E94D80C20914C0130914D01409178
:102E90004E0150914F010E94154B9B01AC012093B4
:102EA000FF023093000340930103509302036091AB
:102EB000FF0270910003809101039091020320E0D2
:102EC00030E048ED51E40E94114B18169CF48091BB
:102ED0009B0290919C02A0919D02B0919E0201964E
:102EE000A11DB11D80939B0290939C02A0939D0213
:102EF000B0939E020E949F0D8091A0019091A1012C
:102F0000A091A201B091A3010196A11DB11D8093D2
:102F1000A0019093A101A093A201B093A30111235A
:102F200009F09CC0419A83E00E94D80C20915C017A
:102F300030915D0140915E0150915F010E94154BFF
:102F40002091C40123FF6EC020E030E040E250E455
:102F50000E945D492DEC3CEC4CEC5DE30E94C649BF
:102F60007B018C016E2D7F2D802F912F2091C5012B
:102F70003091C6014091C7015091C8010E945D493E
:102F80009B01AC01209393023093940240939502ED
:102F900050939602409A85E00E94D80C20915401EB
:102FA0003091550140915601509157010E94154BA7
:102FB0009B01AC01209331023093320240933302E3
:102FC000509334020E94F310A89585E090E090930E
:102FD000AA018093A901809120038160809320033E
:102FE000FF91EF91BF91AF919F918F917F916F91E1
:102FF0005F914F913F912F911F910F91FF90EF9013
:103000000F900BBE0F900FBE0F901F90189510924F
:10301000210210922202109223021092240241985F
:1030200011E0F3CE20E030E040E05FE30E945D4934
:1030300029EA37E848E05EE30E94C6497B018C013B
:103040007F2D912F20E030E0A9010E94C24987FF27
:1030500089CFEE24FF2400E010E084CF80910F039D
:1030600090911003A0911103B09112038093390243
:1030700090933A02A0933B02B0933C0284E00E94FA
:10308000D80C209158013091590140915A0150912A
:103090005B010E94154B20E030E040E05FE30E94BE
:1030A0005D4929EA37E848E05EE30E94C6497B01B2
:1030B0008C017F2D912F20E030E0A9010E94C249B0
:1030C00087FF04C0EE24FF2400E010E06E2D7F2D6A
:1030D000802F912F2091C9013091CA014091CB01DD
:1030E0005091CC010E945D499B01AC0120930F03DC
:1030F00030931003409311035093120313CFEF92B8
:10310000FF920F931F9360910202709103028091CE
:1031100004029091050220E030E0A9010E945E497E
:103120002091060230910702409108025091090255
:103130000E945E4920910A0230910B0240910C02DC
:1031400050910D020E945E4920910E0230910F02B3
:1031500040911002509111020E945E497B018C0146
:1031600020911202309113024091140250911502E5
:10317000CA01B9012E2D3F2D402F512F0E945E49CB
:1031800020E030E040EA50E40E94C6491F910F91D0
:10319000FF90EF900895A091CC028A2F65E00E94E5
:1031A000784BE92FF0E02091930230919402409106
:1031B000950250919602EE0FFF1FEE0FFF1FEE5F7C
:1031C000FD4F2083318342835383AF5FA093CC02B2
:1031D00080918A01882379F08091F50160916001E6
:1031E000982F9F5F9093F5010E94784B992319F4D3
:1031F00081E08093D1010895AF92BF92CF92DF9288
:10320000EF92FF920F931F938091F401982F9F5F8D
:103210009093F4016CE30E94784B992309F46AC1FE
:103220008091D901882309F45AC18091C401837027
:10323000833029F480914601882309F061C180918F
:103240008601909187010197909387018093860171
:103250008091DF019091E00101969093E0018093CD
:10326000DF016091CD017091CE018091CF019091ED
:10327000D00120E030E040E85FE30E945E496093C7
:10328000CD017093CE018093CF019093D0016091D6
:10329000FF0270910003809101039091020320913D
:1032A0000F033091100340911103509112030E94BB
:1032B000154B7B01082FB92E862F9F2DA02FBB2DDC
:1032C00080938B0290938C02A0938D02B0938E0218
:1032D0006E2D7F2D802F9B2D2091C8023091C90229
:1032E0004091CA025091CB020E94114B181664F40F
:1032F0008E2D9F2DA02FBB2D8093C8029093C902C5
:10330000A093CA02B093CB02609131027091320255
:103310008091330290913402209193023091940273
:1033200040919502509196020E94154B162FD72E70
:10333000C82EA92E862F9D2DAC2DBA2D8093030368
:1033400090930403A0930503B0930603612F7D2D92
:103350008C2D9A2D20913502309136024091370202
:10336000509138020E94114B181664F4812F9D2D44
:10337000AC2DBA2D8093350290933602A09337027C
:10338000B093380260911602709117028091180272
:10339000909119022E2D3F2D402F5B2D0E945E49EA
:1033A000609316027093170280931802909319028B
:1033B00060910703709108038091090390910A03BB
:1033C000212F3D2D4C2D5A2D0E945E4960930703FD
:1033D000709308038093090390930A0320910F03CD
:1033E0003091100340911103509112036091250216
:1033F0007091260280912702909128020E945E49D6
:1034000060932502709326028093270290932802EE
:10341000209193023091940240919502509196022E
:1034200060912D0270912E0280912F0290913002B6
:103430000E945E4960932D0270932E0280932F02AA
:10344000909330028091DA019091DB01009739F07E
:1034500001979093DB018093DA01009721F120918D
:10346000E5013091E60121153105A1F040E050E081
:1034700060919702709198028091990290919A02BE
:103480000E94AB4B611571058105910519F481E02E
:103490008093E7011F910F91FF90EF90DF90CF9005
:1034A000BF90AF9008958091DC01882309F447C054
:1034B00081E08093DC018091AF029091B002A091F5
:1034C000B102B091B2020196A11DB11D8093AF026D
:1034D0009093B002A093B102B093B202C0CF6091BA
:1034E00013037091140380911503909116030E94A9
:1034F0002F159BCE81E08093F4010E94CB1890CED3
:1035000080914701882309F49ACE8091C2018823D3
:1035100009F095CE8091A80181508093A80188235D
:1035200009F08DCE81E08093C2010A9A129A83E05D
:103530008093A8018AE091E00E940B4F80CE0E9408
:103540007512B6CF1F920F920FB60F920BB60F9255
:1035500011242F933F934F935F936F937F938F9398
:103560009F93AF93BF93EF93FF938091200382606B
:10357000809320032091A601222341F480E18093CF
:10358000B2008091A7018F5F8093A701809188018D
:1035900090918901181619067CF480918801909108
:1035A0008901019790938901809388018091880116
:1035B00090918901009719F12223D1F08091A70100
:1035C00081508093A701882301F1FF91EF91BF9172
:1035D000AF919F918F917F916F915F914F913F91AB
:1035E0002F910F900BBE0F900FBE0F901F9018954C
:1035F0008091A701813149F71092A70109C080E0AD
:103600000E9413122091A601D7CF80E18093A701D9
:103610008091970290919802A0919902B0919A029C
:103620000196A11DB11D8093970290939802A093DB
:103630009902B0939A020E947E440E94FC188091E5
:10364000210290912202A0912302B09124020196BE
:10365000A11DB11D8093210290932202A093230209
:10366000B09324028091DC01882309F4AECF8091CD
:10367000290290912A02A0912B02B0912C0201966E
:10368000A11DB11D8093290290932A02A0932B02C1
:10369000B0932C029ACFCF93DF938EEA93E02091E0
:1036A000AE033091AF03FC013197A081FC0132974A
:1036B0007081FC0133976081FC013497508105973C
:1036C000EC014881EDB7FEB73E970FB6F894FEBF08
:1036D0000FBEEDBF319681EF90E1CDB7DEB79A8393
:1036E000898333832283A48315827683178260873C
:1036F000118652871386448715860E94EB4EEDB7DC
:10370000FEB73E960FB6F894FEBF0FBEEDBFDF9139
:10371000CF9108952F923F924F925F926F927F9236
:103720008F929F92AF92BF92CF92DF92EF92FF92D1
:103730000F931F93DF93CF93CDB7DEB72B970FB6C1
:10374000F894DEBF0FBECDBFE0901303F0901403DA
:1037500000911503109116032091610130916201CF
:1037600040916301509164018091FF0290910003A8
:10377000A0910103B09102038E839F83A887B9872C
:10378000A0900F03B0901003C0901103D0901203CB
:10379000A0919801B0919901BB87AA8760904801D8
:1037A0007090490180904A0190904B01B091DC01EA
:1037B000B983209031023090320240903302509011
:1037C00034028091930290919402A0919502B0915D
:1037D00096028A839B83AC83BD83ADB7BEB79697B1
:1037E0000FB6F894BEBF0FBEADBFEDB7FEB73196B2
:1037F00061EB70E112967C936E931197E282F382F3
:103800000483158326833783408751878E819F8168
:10381000A885B98582879387A487B587A686B7864A
:10382000C08AD18AAA85BB85B38BA28B648A758A2C
:10383000868A978A8091DF019091E001918F808F35
:103840008091860190918701938F828FB981B48F87
:10385000158E268E378E40A251A28A819B81AC8123
:10386000BD8182A393A3A4A3B5A30E94EB4EADB7E1
:10387000BEB796960FB6F894BEBF0FBEADBF2B96DF
:103880000FB6F894DEBF0FBECDBFCF91DF911F9171
:103890000F91FF90EF90DF90CF90BF90AF909F90EF
:1038A0008F907F906F905F904F903F902F900895F2
:1038B0002F923F924F925F926F927F928F929F9240
:1038C000AF92BF92CF92DF92EF92FF920F931F932E
:1038D000DF93CF93CDB7DEB728970FB6F894DEBF4E
:1038E0000FBECDBFE090F201F090F3010894E11C0F
:1038F000F11CF092F301E092F201C7018F70907019
:10390000009789F4609148017091490180914A01C2
:1039100090914B0120E030E040E252E40E94114BD4
:1039200018160CF485C08091E701882309F098C02F
:103930008091D2019091D30180FD6EC08091D2011F
:103940009091D30182FF09C08091F2019091F3011F
:103950008F709070009709F432C18091D2019091DC
:10396000D30183FF09C08091F2019091F3018F7020
:103970009070009709F46EC18091D2019091D301AB
:1039800084FF04C08091200383FD06C28091D20190
:103990009091D30185FF04C08091200384FD3CC237
:1039A0008091D2019091D30181FF04C080912003C6
:1039B00085FD72C28091D2019091D30181FF04C034
:1039C0008091200386FDDDC08091D2019091D301CA
:1039D00090FF09C08091F2019091F3018F70907077
:1039E000009709F447C028960FB6F894DEBF0FBEC3
:1039F000CDBFCF91DF911F910F91FF90EF90DF909E
:103A0000CF90BF90AF909F908F907F906F905F907E
:103A10004F903F902F9008952FE0E222FF24E11471
:103A2000F10409F08BCF0E944B1B0E948A1B86CFAA
:103A30008091B3029091B402A091B502B091B60208
:103A40000196A11DB11D8093B3029093B402A0937F
:103A5000B502B093B6028091E701882309F468CFDC
:103A60000E948A1B8091A401882309F03FC2109212
:103A7000E70164CF0E944B1BEDB7FEB77A970FB6F4
:103A8000F894FEBF0FBEEDBFEDB6FEB60894E11C84
:103A9000F11C86E79FE092838183609125027091FB
:103AA0002602809127029091280220E030E041E632
:103AB00055E40E94C649D70112966D937D938D936C
:103AC0009C93159760912D0270912E0280912F0288
:103AD0009091300220E030E041E655E40E94C64972
:103AE000F701668377838087918780918B0290911D
:103AF0008C02A0918D02B0918E0282879387A48759
:103B0000B5878091030390910403A0910503B091C0
:103B1000060386879787A08BB18B60911602709100
:103B20001702809118029091190220E030E041E6DE
:103B300055E40E94C649D70152966D937D938D93AB
:103B40009C93559760910703709108038091090336
:103B500090910A0320E030E041E655E40E94C64916
:103B6000F701668B778B808F918F0E94EB4E2DB77C
:103B70003EB7265E3F4F0FB6F8943EBF0FBE2DBF37
:103B800032CF809120038F7B809320038091E101CD
:103B90009091E20100D000D022EA3FE0ADB7BEB77D
:103BA00012963C932E93119714969C938E93139791
:103BB0000E94EB4E0F900F900F900F9005CF0E9438
:103BC0004B1BE0901303F090140300911503109128
:103BD000160320913102309132024091330250910C
:103BE0003402A0909302B0909402C0909502D090BD
:103BF000960280918C0190918D016DB77EB76051D6
:103C000070400FB6F8947EBF0FBE6DBFEDB7FEB724
:103C1000319666E970E1ADB7BEB712967C936E93AC
:103C20001197E282F38204831583268337834087CA
:103C30005187A286B386C486D586978786870E94D9
:103C4000EB4EEDB7FEB770960FB6F894FEBF0FBE01
:103C5000EDBF83CE0E944B1B2091130330911403C0
:103C60004091150350911603E0906101F0906201BC
:103C700000916301109164016090FF027090000355
:103C8000809001039090020320900F033090100366
:103C90004090110350901203609198017091990126
:103CA0007E836D8380918F0290919002A09191020A
:103CB000B091920289839A83AB83BC8360918F0217
:103CC000709190028091910290919202A0900B03CA
:103CD000B0900C03C0900D03D0900E03ADB7BEB7EB
:103CE0005E970FB6F894BEBF0FBEADBFEDB7FEB77F
:103CF0003196F887EF83E0E6F0E11296FC93EE93BD
:103D00001197EF81F8852283338344835583AF81F4
:103D1000B8851696ED92FD920D931C931997EF813D
:103D2000F8856286738684869586AF81B8851E96EF
:103D30002D923D924D925C925197ED81FE8153966A
:103D4000FC93EE93529729813A814B815C81AF813C
:103D5000B88554962D933D934D935C93579720913E
:103D60008A0158962C93589759961C92A601950152
:103D70000E945D49EF81F885628F738F848F958FE4
:103D80000E94EB4E2DB73EB7225E3F4F0FB6F89420
:103D90003EBF0FBE2DBFF0CD0E944B1B40913D0298
:103DA00050913E022091C6023091C70280912103BA
:103DB00090912203A0912303B09124036DB77EB7A5
:103DC0006A5070400FB6F8947EBF0FBE6DBFEDB65F
:103DD000FEB60894E11CF11C6EE270E1EDB7FEB78F
:103DE00072836183F70153834283358324838683FF
:103DF0009783A087B1870E94EB4E80912003877F35
:103E0000809320032DB73EB7265F3F4F0FB6F8943F
:103E10003EBF0FBE2DBFBACD0E944B1B40913D024D
:103E200050913E022091C6023091C7028091210339
:103E300090912203A0912303B09124036DB77EB724
:103E40006A5070400FB6F8947EBF0FBE6DBFEDB6DE
:103E5000FEB60894E11CF11C67EF7FE0EDB7FEB7FA
:103E600072836183F701538342833583248386837E
:103E70009783A087B1870E94EB4E809120038F7EAD
:103E8000809320032DB73EB7265F3F4F0FB6F894BF
:103E90003EBF0FBE2DBF84CD809120038F7D8093C8
:103EA00020032091E1013091E2018091E3019091A2
:103EB000E40100D000D000D0EDB7FEB7319645EC5C
:103EC0005FE0ADB7BEB712965C934E931197338304
:103ED0002283958384830E94EB4EEDB7FEB736961E
:103EE0000FB6F894FEBF0FBEEDBF64CD0E94E9434C
:103EF000BECD0E946B168091F0019091F101019668
:103F00009093F1018093F0018F739070009709F402
:103F100091C06091FF027091000380910103909124
:103F20000203209113033091140340911503509123
:103F300016030E94114B181634F482E090E090931F
:103F40008901809388016091FF0270910003809144
:103F500001039091020320911303309114034091C7
:103F60001503509116030E94C24987FF09C0809132
:103F7000F0019091F1018F779070009709F453C090
:103F800060911303709114038091150390911603AF
:103F900023E333E347E451E40E94114B87FD09C05A
:103FA0008091F0019091F1018F779070009709F462
:103FB00044C0609113037091140380911503909194
:103FC00016032DEC3CEC44E451E40E94114B87FDB8
:103FD00008C08091F0019091F1018F779070009767
:103FE000B1F16091130370911403809115039091C6
:103FF000160323EC35EF40E451E40E94114B87FD9A
:1040000008C08091F0019091F1018F779070009736
:1040100059F18091D2019091D30187FF089581E0F9
:104020000E941312089581E090E09093890180939B
:104030008801A6CF0E94C9136CCF83E00E9413129F
:104040008091D2019091D30187FFE8CFE8CF83E040
:104050000E94131282E00E9413128091D20190916B
:10406000D30187FFDBCFDBCF82E00E941312809168
:10407000D2019091D30187FFD1CFD1CF809120037E
:1040800080FD32C078948091D4019091D501009741
:10409000E9F08091A0019091A101A091A201B091BD
:1040A000A3010097A105B10589F480919401909135
:1040B0009501A0919601B09197010097A105B105D6
:1040C00029F483B7817F866083BF03C083B7817F74
:1040D00083BFF89483B7816083BF7894889583B752
:1040E0008E7F83BF78940895809120038E7F809384
:1040F00020030E94791FC6CF0F931F93CF93DF93A6
:1041000010E00E943F448823A1F18091B003909178
:10411000B1030E947D4EEC018FEFCF3FD80789F3AA
:10412000CD30C9F0C231D10509F444C0CF37D10533
:1041300019F1C830D10501F16091B2037091B30358
:10414000CE010E94BF4EE12FF0E0E353FD4FC0834C
:104150001F5F1133B0F2212F30E0F901E353FD4F1F
:1041600010822F5F3F4FC901DF91CF911F910F91B7
:1041700008950E943E20C5CF112311F410E0C1CF55
:104180006091B2037091B30388E090E00E94BF4E4B
:104190006091B2037091B30380E290E00E94BF4E41
:1041A0006091B2037091B30388E090E00E94BF4E2B
:1041B0001150CFCF6091B2037091B3038DE090E0C6
:1041C0000E94BF4E1123D1F2CDECD2E000E060910D
:1041D000B2037091B303899190E00E94BF4E0F5FCC
:1041E0000117A8F3B6CFEF92FF920F931F93CF93CF
:1041F000DF9300D086E691E1EDB7FEB7928381832D
:104200000E94EB4E0F900F908091B0039091B103FC
:104210000E947C208230910534F08091CD02893754
:1042200049F0893539F0DF91CF911F910F91FF90BF
:10423000EF90089500D0C8ECD1E1EDB7FEB7D2837E
:10424000C1830E94EB4E8CE591E1EDB7FEB79283FE
:1042500081830E94EB4EEDB7FEB7D283C1830E94EB
:10426000EB4E8FEF8093BB028093BC028093BD0224
:104270008093BE028093BF028093C0028093C102EC
:104280008093C2020F900F908BEB92E066E470E097
:1042900049E050E00E94B04F1092D90189ED91E0C1
:1042A00065E370E041E050E00E94B04F11E01093F0
:1042B0008A018AE891E062E470E041E050E00E9407
:1042C000B04F10938B018BE891E063E470E041E024
:1042D00050E00E94B04F0F2EFEEAEF2EF7E4FF2EC3
:1042E000F1EE0F2FFCE31F2FF02DE0924C01F09226
:1042F0004D0100934E0110934F018CE491E060E07A
:1043000070E044E050E00E94B04FE0925001F09223
:104310005101009352011093530180E591E064E054
:1043200070E044E050E00E94B04FE0925401F092FF
:104330005501009356011093570184E591E068E020
:1043400070E044E050E00E94B04F0F2EFAE0EF2EF4
:10435000F7EDFF2EF3EA0F2FFBE31F2FF02DE09276
:104360005801F092590100935A0110935B0188E5BE
:1043700091E06CE070E044E050E00E94B04FE092C9
:104380005C01F0925D0100935E0110935F018CE58A
:1043900091E060E170E044E050E00E94B04F0F2EE9
:1043A000F0E0EF2EF0E0FF2EF0E00F2FF0E01F2FF7
:1043B000F02DE092C501F092C6010093C701109361
:1043C000C80185EC91E064E170E044E050E00E94B7
:1043D000B04FE092C901F092CA010093CB01109353
:1043E000CC0189EC91E068E170E044E050E00E948B
:1043F000B04F83E393E3A3E2B1E480936101909330
:104400006201A0936301B093640181E691E06DE1E4
:1044100070E044E050E00E94B04F0F2EF0E0EF2E2D
:10442000F0E0FF2EF8E50F2FF1E41F2FF02DE092C2
:104430006901F0926A0100936B0110936C0189E6A7
:1044400091E065E270E044E050E00E94B04F86E603
:1044500096E6A6E6B1E480936D0190936E01A09379
:104460006F01B09370018DE691E069E270E044E085
:1044700050E00E94B04F80E090E0AAE7B5E480935E
:10448000820190938301A0938401B093850182E817
:1044900091E06EE370E044E050E00E94B04F80E0B5
:1044A00090E0A0E9B1E48093650190936601A09348
:1044B0006701B093680185E691E061E270E044E055
:1044C00050E00E94B04FE0926101F09262010093CF
:1044D0006301109364010F2EF0E0EF2EF0E0FF2E49
:1044E000F0EA0F2FF0E41F2FF02DE0927101F0920F
:1044F0007201009373011093740181E791E06DE202
:1045000070E044E050E00E94B04FE0927501F092FC
:104510007601009377011093780185E791E061E3DC
:1045200070E044E050E00E94B04F80E090E0A0E4F2
:10453000B1E48093790190937A01A0937B01B093C9
:104540007C0189E791E066E370E044E050E00E947E
:10455000B04F8DEC9CECACE4BFE380937D01909375
:104560007E01A0937F01B09380018DE791E06AE323
:1045700070E044E050E00E94B04F85E0809360011D
:1045800080E691E06CE170E041E050E00E94B04FC5
:104590001092E6011092E50185EE91E064E470E08E
:1045A00042E050E00E94B04FDF91CF911F910F91F8
:1045B000FF90EF9008950E944B1B00D088EC91E192
:1045C000EDB7FEB7928381830E94EB4E0F900F9060
:1045D000089587E59FE00E9409448CE19FE00E94D6
:1045E00009448091A601882389F183E191E000D0FC
:1045F00000D024E13FE0EDB7FEB7328321839483FE
:1046000083830E94EB4E8091BC030F900F900F901C
:104610000F9083FD1EC088E291E000D000D029E019
:104620003FE0EDB7FEB732832183948383830E94FA
:10463000EB4E0F900F9088EC91E1EDB7FEB79283AF
:1046400081830E94EB4E0F900F90089588E191E0D6
:10465000CECF8FE191E0E1CF83E09FE00E9409445B
:104660000895EF92FF920F931F93CF93DF930E94D1
:10467000E92200D08DEF9EE0ADB7BEB712969C93B5
:104680008E9311970E94EB4E0F900F900E94DB22A9
:1046900000D085EF9EE0CDB7DEB79A8389830E9474
:1046A000EB4E0F900F90609197027091980280915D
:1046B000990290919A020E94F10900D08BEE9EE03F
:1046C000EDB7FEB7928381830E94EB4E0F900F905F
:1046D0006091290270912A0280912B0290912C0204
:1046E0000E94F1098091D901882309F4EBC28091DD
:1046F000130390911403A0911503B091160300D0F9
:1047000000D000D025ED3EE0CDB7DEB73A83298357
:10471000EDB7FEB783839483A583B6830E94EB4EE7
:104720002DB73EB72A5F3F4F0FB6F8943EBF0FBE7E
:104730002DBF8091FF0290910003A0910103B091E1
:10474000020300D000D000D02AEA3EE0CDB7DEB7A9
:104750003A832983EDB7FEB783839483A583B68319
:104760000E94EB4E83E99EE0ADB7BEB712969C93D4
:104770008E93119780916D0190916E01A0916F01C0
:10478000B0917001CDB7DEB78B839C83AD83BE83C0
:104790000E94EB4E8CE79EE0EDB7FEB792838183DB
:1047A0008091690190916A01A0916B01B0916C01B7
:1047B000CDB7DEB78B839C83AD83BE830E94EB4E67
:1047C0008091610190916201A0916301B0916401B7
:1047D00026E63EE0EDB7FEB732832183CDB7DEB7E4
:1047E0008B839C83AD83BE830E94EB4E809131020C
:1047F00090913202A0913302B09134022FE43EE056
:10480000EDB7FEB732832183CDB7DEB78B839C83B0
:10481000AD83BE830E94EB4E80910F0390911003F5
:10482000A0911103B09112032AE33EE0EDB7FEB769
:1048300032832183CDB7DEB78B839C83AD83BE8368
:104840000E94EB4E8091930290919402A091950268
:10485000B091960223E23EE0EDB7FEB732832183AA
:10486000CDB7DEB78B839C83AD83BE830E94EB4EB6
:1048700087E09EE0EDB7FEB792838183809171015E
:1048800090917201A0917301B0917401CDB7DEB720
:104890008B839C83AD83BE830E94EB4E8CEE9DE0A8
:1048A000EDB7FEB792838183809175019091760177
:1048B000A0917701B0917801CDB7DEB78B839C834F
:1048C000AD83BE830E94EB4E0F900F900F900F9020
:1048D0008FED9DE0EDB7FEB7928381830E94EB4E92
:1048E0000F900F906091210270912202809123021B
:1048F000909124020E94F10900D000D000D08DEBED
:104900009DE0ADB7BEB712969C938E9311978091A0
:10491000790190917A01A0917B01B0917C01CDB792
:10492000DEB78B839C83AD83BE830E94EB4E809168
:10493000DC01EDB7FEB736960FB6F894FEBF0FBE9A
:10494000EDBF882309F0E4C18091DD01882309F0DF
:10495000D3C100D084E69DE0EDB7FEB7928381839A
:104960000E94EB4E0F900F900E94361200D0C8ECC0
:10497000D1E1ADB7BEB71296DC93CE9311970E94EA
:10498000EB4E0F900F908091DE01882309F0A8C1B3
:1049900000D000D000D08CE19DE0ADB7BEB712963C
:1049A0009C938E93119780917D0190917E01A091AF
:1049B0007F01B0918001EDB7FEB783839483A58317
:1049C000B6830E94EB4E2DB73EB72A5F3F4F0FB61E
:1049D000F8943EBF0FBE2DBF8091D601882309F405
:1049E000BBC08091480190914901A0914A01B091CA
:1049F0004B0100D000D000D026E03DE0EDB7FEB77F
:104A00003283218383839483A583B6830E94EB4EF4
:104A10002DB73EB72A5F3F4F0FB6F8943EBF0FBE8B
:104A20002DBF8091BB028F3F09F480C100D0EDB74C
:104A3000FEB7D283C1830E94EB4E0F900F908091FE
:104A40008A01882309F0C0C000D000D000D08AE0DD
:104A50009CE0CDB7DEB79A83898380916501909100
:104A60006601A0916701B0916801EDB7FEB783833D
:104A70009483A583B6830E94EB4E609102027091ED
:104A80000302809104029091050220E030E0A90128
:104A90000E945E492091060230910702409108026F
:104AA000509109020E945E4920910A0230910B0246
:104AB00040910C0250910D020E945E4920910E021D
:104AC00030910F0240911002509111020E945E49F4
:104AD0007B018C012091120230911302409114024B
:104AE00050911502CDB7DEB72196EBEEFBE0ADB7E6
:104AF000BEB71296FC93EE931197CA01B9012E2D01
:104B00003F2D402F512F0E945E4920E030E040EAC7
:104B100050E40E94C6496A837B838C839D830E94F4
:104B2000EB4E0F900F9083ED9BE0CDB7DEB79A83ED
:104B300089838091E5019091E6019C838B830E949B
:104B4000EB4E0F900F900F900F90DF91CF911F9130
:104B50000F91FF90EF90089500D000D0EDB7FEB711
:104B600031968CEB9CE0ADB7BEB712969C938E93BA
:104B700011978091D701828313820E94EB4E80911E
:104B8000480190914901A0914A01B0914B0100D098
:104B90002BE93CE0CDB7DEB73A832983EDB7FEB70A
:104BA00083839483A583B6830E94EB4E2DB73EB7D3
:104BB0002A5F3F4F0FB6F8943EBF0FBE2DBF8091C6
:104BC0008A01882309F440CF2091E8013091E9015E
:104BD0004091EA015091EB018091EC019091ED013F
:104BE000A091EE01B091EF016DB77EB76A507040B1
:104BF0000FB6F8947EBF0FBE6DBFEDB7FEB731960E
:104C000060E87CE0CDB7DEB77A83698322833383A3
:104C10004483558386839783A087B1870E94EB4E98
:104C200020918B01EDB7FEB73A960FB6F894FEBF10
:104C30000FBEEDBF222309F0AAC040913D02509162
:104C40003E022091C6023091C702809121039091CB
:104C50002203A0912303B0912403CDB7DEB72A9796
:104C60000FB6F894DEBF0FBECDBFEDB7FEB73196DD
:104C700061E47CE07A8369835383428335832483B0
:104C800086839783A087B1870E94EB4E20916001B5
:104C9000EDB7FEB736960FB6F894FEBF0FBEEDBF68
:104CA000319685E29CE0ADB7BEB712969C938E9389
:104CB0001197228313820E94EB4E0F900F900F905A
:104CC0000F90C2CE8091130390911403A09115030D
:104CD000B091160300D000D000D02FEB3EE014CDF1
:104CE00000D084E49DE0EDB7FEB7928381830E94FB
:104CF000EB4E0F900F904CCE00D08CE79DE0CDB7DF
:104D0000DEB79A8389830E94EB4E0F900F9021CEDD
:104D100000D08BE99DE0ADB7BEB712969C938E9301
:104D200011970E94EB4E0F900F900ECE8091BC0217
:104D30008F3F09F07BCE8091BD028F3F09F076CE88
:104D40008091BE028F3F09F071CE8091BF028F3FEC
:104D500009F06CCE8091C0028F3F09F067CE809140
:104D6000C1028F3F09F062CE8091C2028F3F09F0ED
:104D70005DCE00D085ED9CE0ADB7BEB712969C939A
:104D80008E9311970E94EB4E0F900F904FCE00D054
:104D900000D0EDB7FEB7319680E79CE0ADB7BEB767
:104DA00012969C938E931197228313820E94EB4E4E
:104DB0000F900F900F900F9040CFEF92FF920F93B4
:104DC0001F93CF93DF938091130390911403A091CD
:104DD0001503B091160300D000D000D02AEA3BE0C2
:104DE000EDB7FEB73283218383839483A583B68393
:104DF0000E94EB4E8DB79EB706960FB6F8949EBFF5
:104E00000FBE8DBF8091B0039091B1030E947C20B2
:104E1000823050F18DEC92E00E94124DE09013032D
:104E2000F090140300911503109116032091500186
:104E30003091510140915201509153010E94154B04
:104E4000A80197010E94C6496093500170935101D7
:104E5000809352019093530180E591E064E070E00B
:104E600044E050E00E94B04F00D0C8ECD1E1EDB773
:104E7000FEB7D283C1830E94EB4E8091FF029091D6
:104E80000003A0910103B091020300D000D023E8F9
:104E90003BE0EDB7FEB73283218383839483A58300
:104EA000B6830E94EB4E8DB79EB706960FB6F89468
:104EB0009EBF0FBE8DBF8091B0039091B1030E9441
:104EC0007C20823050F18DEC92E00E94124DE090F7
:104ED000FF02F09000030091010310910203209162
:104EE0004C0130914D0140914E0150914F010E9473
:104EF000154BA80197010E94C64960934C0170931D
:104F00004D0180934E0190934F018CE491E060E05D
:104F100070E044E050E00E94B04F00D0EDB7FEB723
:104F2000D283C1830E94EB4E809131029091320274
:104F3000A0913302B091340200D000D02DE53BE0C7
:104F4000EDB7FEB73283218383839483A583B68331
:104F50000E94EB4E8DB79EB706960FB6F8949EBF93
:104F60000FBE8DBF8091B0039091B1030E947C2051
:104F7000823050F18DEC92E00E94124DE0903102AF
:104F8000F0903202009133021091340220915401CA
:104F90003091550140915601509157010E94154B97
:104FA000A80197010E94C64960935401709355016E
:104FB000809356019093570184E591E068E070E09A
:104FC00044E050E00E94B04F00D0EDB7FEB7D2836E
:104FD000C1830E94EB4E8091930290919402A09124
:104FE0009502B091960200D000D027E33BE0EDB7E8
:104FF000FEB73283218383839483A583B6830E9483
:10500000EB4E8DB79EB706960FB6F8949EBF0FBEB7
:105010008DBF8091B0039091B1030E947C208230BB
:1050200060F18DEC92E00E94124D9B01AC01609109
:1050300093027091940280919502909196020E9441
:105040005D499B01AC016091C5017091C6018091E1
:10505000C7019091C8010E945E496093C501709399
:10506000C6018093C7019093C80185EC91E064E18B
:1050700070E044E050E00E94B04F00D0EDB7FEB7C2
:10508000D283C1830E94EB4E80910F039091100355
:10509000A0911103B091120300D000D023E13BE0B6
:1050A000EDB7FEB73283218383839483A583B683D0
:1050B0000E94EB4E8DB79EB706960FB6F8949EBF32
:1050C0000FBE8DBF8091B0039091B1030E947C20F0
:1050D000823060F18DEC92E00E94124D9B01AC0198
:1050E00060910F037091100380911103909112034E
:1050F0000E945D499B01AC016091C9017091CA0198
:105100008091CB019091CC010E945E496093C901CE
:105110007093CA018093CB019093CC0189EC91E00C
:1051200068E170E044E050E00E94B04F00D0EDB77D
:10513000FEB7D283C1830E94EB4E0F900F90DF9198
:10514000CF911F910F91FF90EF900895CF93DF9330
:1051500000D000D000D08AEE9AE0EDB7FEB792837F
:1051600081838091690190916A01A0916B01B09156
:105170006C0183839483A583B6830E94EB4E8DB725
:105180009EB706960FB6F8949EBF0FBE8DBF809156
:10519000B0039091B1030E947C208230A0F08DEC8E
:1051A00092E00E94124D6093690170936A018093AE
:1051B0006B0190936C0189E691E065E270E044E058
:1051C00050E00E94B04F00D0C8ECD1E1EDB7FEB77F
:1051D000D283C1830E94EB4E00D000D081EC9AE0D4
:1051E000EDB7FEB79283818380916D0190916E013E
:1051F000A0916F01B091700183839483A583B683DE
:105200000E94EB4E8DB79EB706960FB6F8949EBFE0
:105210000FBE8DBF8091B0039091B1030E947C209E
:105220008230A0F08DEC92E00E94124D60936D01EF
:1052300070936E0180936F01909370018DE691E001
:1052400069E270E044E050E00E94B04F00D0EDB75A
:10525000FEB7D283C1830E94EB4E80916901909189
:105260006A01A0916B01B0916C01809361019093F0
:105270006201A0936301B09364010F900F90DF91DE
:10528000CF91089584EB9AE00E94094486EA9AE05F
:105290000E9409448AE89AE00E9409448FE69AE055
:1052A0000E9409448CE49AE00E94094480E39AE059
:1052B0000E9409448AE09AE00E9409448BEE99E03A
:1052C0000E94094488EC99E00E94094483EB99E02C
:1052D0000E94094487E999E00E9409448DE799E01A
:1052E0000E94094482E699E00E9409448DE399E016
:1052F0000E94094483E299E00E940944089500D085
:1053000086E199E0EDB7FEB7928381830E94EB4E70
:105310008091A4010F900F90882309F408950E94B2
:10532000E943089589E099E00E94094481EF98E0FB
:105330000E9409448AED98E00E9409448CEC98E0B0
:105340000E9409448AEB98E00E94094485EA98E0AB
:105350000E9409448AE898E00E94094489E798E09D
:105360000E9409448AE698E00E9409448AE598E090
:105370000E9409448CE398E00E9409448BE198E084
:105380000E9409448CEF97E00E9409448AED97E05F
:105390000E9409448091C40182FF17C08091C3011B
:1053A000882309F495C082E391E000D000D028EC76
:1053B00037E0EDB7FEB732832183948383830E9465
:1053C000EB4E0F900F900F900F9080918A018823E1
:1053D00009F075C08FE291E000D000D025EB37E0F6
:1053E000EDB7FEB732832183948383830E94EB4E13
:1053F0000F900F900F900F9080918B01882309F0F0
:105400005BC08FE291E000D000D02AE937E0EDB731
:10541000FEB732832183948383830E94EB4E0F90E7
:105420000F908CE797E0EDB7FEB7928381830E94DF
:10543000EB4E0F900F9088E697E00E94094487E4B6
:1054400097E00E94094488E297E00E940944809115
:10545000C40180FF18C0809146018823B1F182E326
:1054600091E000D000D022E137E0EDB7FEB7328303
:105470002183948383830E94EB4E8091C4010F901B
:105480000F900F900F9081FF16C0809147018823E5
:10549000C9F082E391E000D000D025EF36E0EDB70F
:1054A000FEB732832183948383830E94EB4E0F9057
:1054B0000F900F900F90089582E391E0A4CF82E3C4
:1054C00091E08ACF8FE291E0E6CF8FE291E0C9CF01
:1054D0008FE291E06ACF2F923F924F925F926F924C
:1054E0007F928F929F92AF92BF92CF92DF92EF9274
:1054F000FF920F931F93CF93DF93822E732E642E10
:10550000552E462E372E282E992E263609F48EC07B
:10551000282D372D462D552D642D732D822D992D37
:1055200006E6A02E16E6B12ECC24DD24EE24FF24C0
:1055300000E010E00E946B458230E0F1882D893652
:1055400009F4ADC3282D372D462D552D642D732D0F
:10555000822D992DF9E6AF2EE4E7BE2ECC24DD2472
:10556000EE24FF2400E010E00E946B45823008F03A
:10557000F1C0E82DE83609F4D8C1882D853609F444
:105580009BC1E82DE63709F44AC10E947F29DF91CB
:10559000CF911F910F91FF90EF90DF90CF90BF9030
:1055A000AF909F908F907F906F905F904F903F90C3
:1055B0002F900895882D8C3609F4DCC3282D372DC3
:1055C000462D552D642D732D822D992DBCE6AB2EC5
:1055D000A1E6BA2ECC24DD24EE24FF2400E010E066
:1055E0000E946B45823008F08BC0E82DED3609F43F
:1055F00006C2F82DF93609F4F9C2982D983629F625
:10560000772019F6662009F6552009F0BECF442010
:1056100009F0BBCF332009F0B8CF222009F0B5CF75
:10562000992009F0B2CF0E944229B1CF363609F055
:105630006FCF442309F06CCF552309F069CF66235F
:1056400009F066CF772309F063CF882309F060CF94
:10565000992309F05DCF8091A501882309F495CFA6
:1056600000D08BE796E0EDB7FEB7928381830E946E
:10567000EB4E00D000D08DE596E0EDB7FEB79283FB
:1056800081838091820190918301A0918401B091E6
:10569000850183839483A583B6830E94EB4E8DB7E7
:1056A0009EB706960FB6F8949EBF0FBE8DBF809131
:1056B000B0039091B1030E947C2082309105A4F048
:1056C0008DEC92E00E94124D6093820170938301F1
:1056D000809384019093850182E891E06EE370E00D
:1056E00044E050E00E94B04F00D088EC91E1EDB76B
:1056F000FEB7928381830E94EB4E0F900F9047CFAD
:10570000E82DE13609F454C2882D863709F4F7C133
:10571000E82DE13609F039CFF72DF23609F035CF13
:10572000662009F032CF552009F02FCF442009F030
:105730002CCF332009F029CF222009F026CF992041
:1057400009F023CF8091A501882309F41ECF0E9480
:10575000A6281DCF882D8C3609F478C1E82DE037B6
:1057600009F467C1E82DE73609F00FCFF72DF637BA
:1057700009F00BCF662009F008CF552009F005CFBE
:10578000442009F002CF332009F0FFCE222009F097
:10579000FCCE992009F0F9CE8091A501882309F467
:1057A000F4CE8091610190916201A0916301B0916A
:1057B000640100D000D000D023E436E0EDB7FEB79E
:1057C0003283218383839483A583B6830E94EB4E27
:1057D0008DB79EB706960FB6F8949EBF0FBE8DBFCD
:1057E0008091B0039091B1030E947C20823091059A
:1057F0000CF47ACF8DEC92E00E94124D609361011F
:1058000070936201809363019093640181E691E05B
:105810006DE170E044E050E00E94B04F65CFF72D9D
:10582000F63609F0B2CE662009F0AFCE552009F069
:10583000ACCE442009F0A9CE332009F0A6CE222018
:1058400009F0A3CE992009F0A0CE81E09091D90172
:10585000911180E08093D901882309F4E4C286E3A2
:1058600091E000D000D025ED36E0EDB7FEB73283F1
:105870002183948383830E94EB4E0F900F900F90AF
:105880000F908091D901882309F0D0C289ED91E071
:1058900065E370E041E050E00E94B04F8091D90193
:1058A000882309F474CE81E691E06DE170E044E074
:1058B00050E00E94A04F6BCE972D943709F065CE33
:1058C000662009F062CE552009F05FCE442009F031
:1058D0005CCE332009F059CE222009F056CE992013
:1058E00009F053CE8091A501882309F44ECE0E9481
:1058F000C9138091480190914901A0914A01B0914A
:105900004B0100D000D000D02BE835E0EDB7FEB75A
:105910003283218383839483A583B6830E94EB4ED5
:105920000F900F900F900F90E0CEF72DF23709F007
:105930002CCE662009F029CE552009F026CE442031
:1059400009F023CE332009F020CE222009F01DCE0D
:10595000992009F01ACE8091A501882309F415CE6B
:1059600000D000D000D080EA95E0EDB7FEB792837A
:10597000818380917D0190917E01A0917F01B09102
:10598000800183839483A583B6830E94EB4E8DB7F9
:105990009EB706960FB6F8949EBF0FBE8DBF80913E
:1059A000B0039091B1030E947C20823091050CF4E9
:1059B0009BCE60917D0170917E0180917F019091DD
:1059C00080012DEC3CEC4CEC5DE30E94114B181671
:1059D0000CF08ACE8DEC92E00E94124D60937D0116
:1059E00070937E0180937F01909380018DE791E019
:1059F0006AE370E044E050E00E94B04F75CE77203B
:105A000009F0C3CD662009F0C0CD552009F0BDCD09
:105A1000442009F0BACD332009F0B7CD222009F097
:105A2000B4CD992009F0B1CD1092D8010E949229ED
:105A3000AECDF72DFC3609F0A8CD862D853609F0C0
:105A4000A4CD952D983609F0A0CDE1CD972D9637B0
:105A500009F09BCD662009F098CD552009F095CD31
:105A6000442009F092CD332009F08FCD222009F097
:105A70008CCD992009F089CD8091A501882309F466
:105A800084CD00D000D000D084E296E0EDB7FEB720
:105A9000928381838091650190916601A091670155
:105AA000B091680183839483A583B6830E94EB4EF3
:105AB0008DB79EB706960FB6F8949EBF0FBE8DBFEA
:105AC0008091B0039091B1030E947C2082309105B7
:105AD0000CF40ACE8DEC92E00E94124D60936501A9
:105AE00070936601809367019093680185E691E069
:105AF00061E270E044E050E00E94B04FF5CD972D98
:105B0000943609F042CD662009F03FCD552009F0CA
:105B10003CCD442009F039CD332009F036CD222088
:105B200009F033CD992009F030CD8091A50188236B
:105B300009F42BCD00D000D000D08EEB95E0EDB76E
:105B4000FEB7928381838091790190917A01A0912F
:105B50007B01B0917C0183839483A583B6830E94EB
:105B6000EB4E8DB79EB706960FB6F8949EBF0FBE4C
:105B70008DBF8091B0039091B1030E947C20823050
:105B800091050CF4B1CD8DEC92E00E94124D609322
:105B9000790170937A0180937B0190937C0189E76E
:105BA00091E066E370E044E050E00E94B04F9CCD8D
:105BB000F72DF33609F0B0CD662009F0E6CC55207C
:105BC00009F0E3CC442009F0E0CC332009F0DDCC2F
:105BD000222009F0DACC992009F0D7CC8091A501D8
:105BE000882309F4D2CC0E94DD26D1CC872D8136C2
:105BF00009F0CBCC662009F0C8CC552009F0C5CC03
:105C0000442009F0C2CC332009F0BFCC222009F097
:105C1000BCCC992009F0B9CC8091A501882309F466
:105C2000B4CC00D000D000D08DEF95E0EDB7FEB73A
:105C3000928381838091710190917201A09173018F
:105C4000B091740183839483A583B6830E94EB4E45
:105C50008DB79EB706960FB6F8949EBF0FBE8DBF48
:105C60008091B0039091B1030E947C208230910515
:105C70000CF43ACD8DEC92E00E94124D60937101CC
:105C800070937201809373019093740181E791E0A6
:105C90006DE270E044E050E00E94B04F25CD972DBA
:105CA000943709F04FCC662009F04CCC552009F010
:105CB00049CC442009F046CC332009F043CC2220C3
:105CC00009F040CC992009F03DCC8091A5018823B2
:105CD00009F45BCC0E94700B00D0C8ECD1E1EDB7A9
:105CE000FEB7D283C1830E94EB4E8BE695E0EDB701
:105CF000FEB7928381830E94EB4E0F900F908091AC
:105D0000B0039091B1030E947C20823091053CF059
:105D10008DEC92E00E94164D883008F4AFC000D0A0
:105D2000EDB7FEB7D283C1830E94EB4E8AE495E0C3
:105D3000EDB7FEB7928381830E94EB4E0F900F90D8
:105D40008091B0039091B1030E947C208230910534
:105D50003CF08DEC92E00E94164D883008F472C041
:105D600000D0EDB7FEB7D283C1830E94EB4E0F90F7
:105D70000F900DCC972D913609F020CC662009F0BC
:105D80001DCC552009F01ACC442009F017CC332043
:105D900009F014CC222009F011CC992009F00ECC86
:105DA0008091A501882309F4F0CB00D000D000D069
:105DB00087ED95E0EDB7FEB7928381838091750101
:105DC00090917601A0917701B091780183839483BB
:105DD000A583B6830E94EB4E8DB79EB706960FB68D
:105DE000F8949EBF0FBE8DBF8091B0039091B10318
:105DF0000E947C20823091050CF476CC8DEC92E0F0
:105E00000E94124D60937501709376018093770123
:105E10009093780185E791E061E370E044E050E021
:105E20000E94B04F61CC89E391E01BCD00D084EBA0
:105E300096E0EDB7FEB7928381830E94EB4E0F9000
:105E40000F9024CD90E0FC01EE0FFF1FEE0FFF1F1F
:105E5000EE0FFF1FE80FF91FA7E1B3E0E15CFD4F74
:105E600089E001900D928150E1F787E193E06FE4C2
:105E700070E049E050E00E94B04F72CF90E0FC012A
:105E8000EE0FFF1FEE0FFF1FEE0FFF1FE80FF91FB2
:105E9000ABEBB2E0E15CFD4F89E001900D928150E7
:105EA000E1F78BEB92E066E470E049E050E00E949D
:105EB000B04F35CF2F923F924F925F926F927F9269
:105EC0008F929F92AF92BF92CF92DF92EF92FF920A
:105ED0000F931F93DF93CF93CDB7DEB72C970FB6F9
:105EE000F894DEBF0FBECDBF822E732E642E552ECA
:105EF000462E372E282E992E233709F446C1282DF9
:105F0000372D462D552D642D732D822D992D03E7A8
:105F1000A02E13E7B12ECC24DD24EE24FF2400E0D4
:105F200010E00E946B45823008F4D4C0282D213344
:105F300009F47FC5282D372D462D552D642D732D41
:105F4000822D992DB1E3AB2EA1E3BA2EF1E7CF2E2E
:105F5000DD24EE24FF2400E010E00E946B45823037
:105F600008F032C1782D723709F408C5282D372D75
:105F7000462D552D642D732D822D992DE2E7AE2EE1
:105F800002E7B02E15E6C12EDD24EE24FF2400E04A
:105F900010E00E946B45823008F408C2F82DF537F6
:105FA00009F4A8C6682D603309F033C1772D713329
:105FB00009F02FC1862D813709F02BC1552009F03A
:105FC00028C1442009F025C1332009F022C1222034
:105FD00009F01FC1992009F01CC100D08DE793E0A2
:105FE000ADB7BEB712969C938E9311970E94EB4E5D
:105FF000EDB7FEB77C970FB6F894FEBF0FBEEDBFAE
:1060000031968BE493E0ADB7BEB712969C938E9316
:10601000119780919B0290919C02A0919D02B0915A
:106020009E0282839383A483B58380919F02909183
:10603000A002A091A102B091A20286839783A087BB
:10604000B1878091A3029091A402A091A502B09182
:10605000A60282879387A487B5878091A702909133
:10606000A802A091A902B091AA0286879787A08B67
:10607000B18B8091AB029091AC02A091AD02B09136
:10608000AE02828B938BA48BB58B8091B3029091DF
:10609000B402A091B502B091B602868B978BA08F07
:1060A000B18F8091AF029091B002A091B102B091F6
:1060B000B202828F938FA48FB58F0E94EB4EEDB703
:1060C000FEB77E960FB6F894FEBF0FBEEDBF21E07F
:1060D00030E0A1C0282D203309F485C4282D372DA8
:1060E000462D552D642D732D822D992DB0E3AB2EA9
:1060F000A1E7BA2ECC24DD24EE24FF2400E010E03A
:106100000E946B45823008F0A0C0682D603709F40A
:10611000F0C3282D372D462D552D642D732D822D3E
:10612000992DF0E7AF2EECE6BE2ECC24DD24EE2434
:10613000FF2400E010E00E946B45823008F4B8C1F3
:10614000A82DA93609F424C6E82DE73709F061C067
:10615000F72DFF3609F05DC0662009F05AC05520C2
:1061600009F057C0442009F054C0332009F051C051
:10617000222009F04EC0992009F04BC00E94700BFC
:106180008091A4018823E9F04FC4333709F0B7CEDA
:10619000442309F0B4CE552309F0B1CE662309F0AB
:1061A000AECE772309F0ABCE882309F0A8CE992391
:1061B00009F0A5CE0E9431238091A401882309F023
:1061C00033C421E030E027C0982D943709F4EEC3A2
:1061D000282D372D462D552D642D732D822D992D6B
:1061E000B4E7AB2EAFE6BA2EFFE6CF2EE2E6DE2E08
:1061F000EE24FF2400E010E00E946B45823008F09E
:106200008AC0F82DF03709F42BC5782D733709F4BF
:10621000E1C420E030E0C9012C960FB6F894DEBF4F
:106220000FBECDBFCF91DF911F910F91FF90EF90E7
:10623000DF90CF90BF90AF909F908F907F906F90A6
:106240005F904F903F902F900895282D233309F4AD
:10625000FBC2282D372D462D552D642D732D822DF3
:10626000992D03E3A02E11E7B12ECC24DD24EE24DA
:10627000FF2400E010E00E946B45823008F40DC25C
:10628000A82DA43309F469C5E82DE03311F6F72DE4
:10629000F23709F0BECF662009F0BBCF552009F0D8
:1062A000B8CF442009F0B5CF332009F0B2CF222077
:1062B00009F0AFCF992009F0ACCF1092D301109222
:1062C000D2018091B0039091B1030E947C20823072
:1062D00091050CF4FDC58DEC92E00E94124D0E94D8
:1062E0002E4A8B018091B0039091B1030E947C20D3
:1062F0008230910554F08DEC92E00E94124D0E9484
:106300002E4A0617170709F40DC68091A4018823A9
:1063100009F457CF89C3B82DB93609F492C5382D81
:10632000323709F076CF672D673609F072CF762DB8
:10633000703709F06ECF852D853709F06ACF44207C
:1063400009F067CF332009F064CF222009F061CF34
:10635000992009F05ECF00D086E492E0ADB7BEB7D9
:1063600012969C938E9311970E94EB4E0F900F9074
:106370008091A4010E94E94388E10FB6F8948093CC
:106380006000109260000FBE83ED9CE1FC01E115FE
:10639000F10511F03197F1F78115910511F0019791
:1063A000F1F70C94007C21E030E035CFA82DA83720
:1063B00009F02FCFB72DB43709F02BCFE62DE136FA
:1063C00009F027CF552009F024CF442009F021CF30
:1063D000332009F01ECF222009F01BCF992009F0AD
:1063E00018CF8091C40180FFABC381FFA9C3809106
:1063F0004701882309F490C586E391E000D000D0DE
:1064000023EB32E0ADB7BEB712963C932E931197B3
:1064100014969C938E9313970E94EB4E80914601A5
:106420000F900F900F900F90882309F472C586E3A8
:1064300091E000D000D023EA32E0EDB7FEB732831E
:106440002183948383830E94EB4E0F900F900F90D3
:106450000F90019B5BC586E391E000D000D02FE850
:1064600032E0ADB7BEB712963C932E9311971496B7
:106470009C938E9313970E94EB4E0F900F900F906A
:106480000F9002994CC522E431E000D000D08BE798
:1064900092E0EDB7FEB792838183348323830E9419
:1064A000EB4E0F900F900F900F9021E030E0B3CEA5
:1064B000882D853609F0ADCE972D943609F0A9CEFA
:1064C000662009F0A6CE552009F0A3CE442009F09D
:1064D000A0CE332009F09DCE222009F09ACE99203B
:1064E00009F097CE8091A501882309F429C300D033
:1064F00000D08DE395E0EDB7FEB79283818381E014
:1065000090E0948383830E94EB4E8EE295E0ADB7DA
:10651000BEB712969C938E93119782E090E01496EA
:106520009C938E9313970E94EB4E81E295E0EDB71A
:10653000FEB79283818384E090E0948383830E94FA
:10654000EB4E84E195E0ADB7BEB712969C938E9367
:10655000119788E090E014969C938E9313970E9475
:10656000EB4E82E095E0EDB7FEB79283818380E148
:1065700090E0948383830E94EB4E8BEE94E0ADB762
:10658000BEB712969C938E93119780E290E014967A
:106590009C938E9313970E94EB4E80EE94E0EDB7A0
:1065A000FEB79283818380E490E0948383830E948A
:1065B000EB4E84ED94E0ADB7BEB712969C938E93EC
:1065C000119780E890E014969C938E9313970E9405
:1065D000EB4E86EC94E0EDB7FEB79283818380E0CA
:1065E00091E0948383830E94EB4E8091D20190913D
:1065F000D3012CEA34E0ADB7BEB712963C932E938C
:10660000119714969C938E9313970E94EB4E0F90C4
:106610000F900F900F908091B0039091B1030E9462
:106620007C208230910564F08DEC92E060E070E0B7
:1066300040E150E00E94044C7093D3016093D2017A
:1066400000D088EC91E1EDB7FEB7928381830E9480
:10665000EB4E8091D2019091D3010F900F9080FD6D
:1066600072C48091D2019091D30190FD60C4809159
:10667000D2019091D30183FFA4CD00D088EC93E0A8
:10668000ADB7BEB712969C938E9311970E94EB4EB6
:106690000F900F9021E030E0BECD682D613309F4FA
:1066A00041C3882D823309F0B4CD972D913709F07D
:1066B000B0CD662009F0ADCD552009F0AACD44201B
:1066C00009F0A7CD332009F0A4CD222009F0A1CDF7
:1066D000992009F09ECD1092D3011092D2018090A2
:1066E000130390901403A0901503B090160320910B
:1066F00061013091620140916301509164016091A8
:10670000FF02709100038091010390910203698759
:106710007A878B879C8740900F035090100360907E
:10672000110370901203E0904801F090490100912C
:106730004A0110914B013090DC018091310290911F
:106740003202A0913302B091340289839A83AB83E1
:10675000BC83609193027091940280919502909114
:1067600096026D837E838F8398878DB79EB78C97B3
:106770000FB6F8949EBF0FBE8DBFEDB7FEB7319632
:1067800066EC71E0ADB7BEB712967C936E9311972D
:1067900082829382A482B582268337834087518781
:1067A00069857A858B859C856287738784879587C1
:1067B00046865786608A718AE28AF38A048B158B33
:1067C0008091790190917A01A0917B01B0917C0137
:1067D000868B978BA08FB18F80917D0190917E01E8
:1067E000A0917F01B0918001828F938FA48FB58F8C
:1067F0008091DD01868F178E30A211A28091DA017F
:106800009091DB0193A382A389819A81AB81BC81A2
:1068100084A395A3A6A3B7A36D817E818F8198855C
:1068200060A771A782A793A70E94EB4E8091A40155
:10683000ADB7BEB79C960FB6F894BEBF0FBEADBF46
:10684000882309F4BECCF0C0372D313709F001CDD3
:10685000662009F0FECC552009F0FBCC442009F05D
:10686000F8CC332009F0F5CC222009F0F2CC9920A5
:1068700009F0EFCC1092D3011092D20120911303B2
:1068800030911403409115035091160380919302A7
:1068900090919402A0919502B0919602EDB7FEB747
:1068A0003A970FB6F894FEBF0FBEEDBFEDB6FEB639
:1068B0000894E11CF11C67EB71E072836183F701BE
:1068C000228333834483558386839783A087B1874C
:1068D0000E94EB4E8091A4012DB73EB7265F3F4F3B
:1068E0000FB6F8943EBF0FBE2DBF882309F469CCC4
:1068F0009BC0772D7C3609F00CCC662009F009CCC2
:10690000552009F006CC442009F003CC332009F0CF
:1069100000CC222009F0FDCB992009F0FACB809120
:10692000C40182FF0DC19091C30181E0911180E00B
:106930008093C3018091C301882309F4DAC226E35E
:1069400031E000D000D08EE092E0ADB7BEB7129635
:106950009C938E93119714963C932E9313970E94B9
:10696000EB4E8091C3010F900F900F900F908823F2
:1069700009F4BBC25F9A21E030E04DCC872D82370D
:1069800009F0F4CA962D953609F0F0CA552009F0A1
:10699000EDCA442009F0EACA332009F0E7CA2220F0
:1069A00009F0E4CA992009F418CBE0CAA72DAF3644
:1069B00009F00ECCB62DBF3609F00ACCE52DE23633
:1069C00009F006CC442009F003CC332009F000CCB8
:1069D000222009F0FDCB992009F0FACB0C9400009D
:1069E00021E030E018CC372D313709F077CB662025
:1069F00009F074CB552009F071CB442009F06ECB1F
:106A0000332009F06BCB222009F068CB992009F0E4
:106A100065CB1092D3011092D2010E942C23809159
:106A2000A401882309F4CDCB0E94E94321E030E0A2
:106A3000F2CB372D313309F07DCA662D613709F06D
:106A400079CA552009F076CA442009F073CA332068
:106A500009F070CA222009F06DCA992009F06ACAAB
:106A6000F89449E021E030E0F90140935700C895DF
:106A7000E02C20E030E0F90140935700C895902CBD
:106A80007894F89423E030E0F90140935700C895DA
:106A9000802C82E090E0FC0140935700C895702C58
:106AA000789400D000D000D041E453E0ADB7BEB739
:106AB00012965C934E931197809187029091880271
:106AC000A0918902B0918A02EDB7FEB783839483C7
:106AD000A583B6830E94EB4E00D000D0EDB7FEB781
:106AE00031964AE153E0ADB7BEB712965C934E9330
:106AF0001197728213828482158296821782E086B1
:106B000011860E94EB4EEDB7FEB73A960FB6F89499
:106B1000FEBF0FBEEDBFEDEBF3E020E4EF3FF20769
:106B200009F098F480E090E005C030E4EF3FF3070F
:106B300009F068F431962081253CB9F70196F5CF2C
:106B40000E947F2921E030E066CB80E090E000D019
:106B500000D028E033E0ADB7BEB712963C932E9339
:106B6000119714969C938E9313970E94EB4E20914D
:106B70006600EDB7FEB731968CEF92E0ADB7BEB7C9
:106B800012969C938E931197228313820E94EB4E50
:106B90008091C4009091C50021EF32E0EDB7FEB7BF
:106BA00032832183948383830E94EB4E0F900F9056
:106BB00088EC91E1ADB7BEB712969C938E93119776
:106BC0000E94EB4E8091A4010F900F90882309F44E
:106BD000F8CA2ACF872D883709F01BCB962D94371A
:106BE00009F017CBA52DA13609F013CB442009F0ED
:106BF00010CB332009F00DCB222009F00ACB9920CD
:106C000009F007CB8091C40181FF9ACF9091470191
:106C100081E0911180E080934701809147018823B2
:106C200009F460C126E331E000D000D08AE492E0AC
:106C3000EDB7FEB792838183348323830E94EB4EAA
:106C4000809147010F900F900F900F90882309F4C7
:106C500042C181E090E00E94950A21E030E0DBCA69
:106C6000272D283709F0D5CA362D343709F0D1CA77
:106C7000652D613609F0CDCA442009F0CACA332017
:106C800009F0C7CA222009F0C4CA992009F0C1CA74
:106C90008091C40180FF54CF9091460181E0911111
:106CA00080E08093460180914601882309F42BC13E
:106CB00026E331E000D000D084E692E0ADB7BEB765
:106CC00012969C938E93119714963C932E93139740
:106CD0000E94EB4E809146010F900F900F900F9005
:106CE000882309F409C181E090E00E94840A21E030
:106CF00030E091CA272D233609F08BCA362D3D3658
:106D000009F087CA552009F084CA442009F081CAD5
:106D1000332009F07ECA222009F07BCA992009F0AD
:106D200078CA9ECE772D713709F073CA662009F0B4
:106D300070CA552009F06DCA442009F06ACA332090
:106D400009F067CA222009F064CA992009F061CAD3
:106D50001092D3011092D2012DCAB72DB13709F08C
:106D600058CA662009F055CA552009F052CA442075
:106D700009F04FCA332009F04CCA222009F049CA51
:106D8000992009F046CA1092D3011092D201F6C997
:106D9000B72DBD3609F03DCA662009F03ACA552024
:106DA00009F037CA442009F034CA332009F031CA47
:106DB000222009F02ECA992009F02BCA8091A50142
:106DC000882309F4BDCE2091600100D000D0EDB73A
:106DD000FEB731968FE192E0ADB7BEB712969C93A5
:106DE0008E931197228313820E94EB4E0F900F9087
:106DF0000F900F908091B0039091B1030E947C207E
:106E00008230910584F08DEC92E00E94124D0E9438
:106E1000334A6093600180E691E06CE170E041E00C
:106E200050E00E94B04F00D088EC91E1EDB7FEB782
:106E3000928381830E94EB4E0F900F9021E030E00F
:106E4000EAC9E72DE33609F0E4C9F62DF33709F076
:106E5000E0C9252D2F3609F0DCC9442009F0D9C935
:106E6000332009F0D6C9222009F0D3C9992009F0AE
:106E7000D0C98091A501882309F462CE20916600D3
:106E800000D000D0EDB7FEB7319683EC92E0ADB7FD
:106E9000BEB712969C938E931197228313820E9401
:106EA000EB4E0F900F900F900F908091B003909148
:106EB000B1030E947C20823091050CF4B4CF8DEC9C
:106EC00092E00E94124D0E94334A60936600ABCF5D
:106ED0000FEF1FEF07CA80E090E00E94950A21E0C3
:106EE00030E099C929E331E09FCE5F9821E030E09E
:106EF00092C929E331E025CD80E090E00E94840A28
:106F000021E030E088C929E331E0D4CE89E391E083
:106F1000A4CA89E391E08DCA89E391E06FCA2DE3A9
:106F200031E0B3CA1093DB010093DA01EEC900D05F
:106F300084E194E0EDB7FEB7928381830E94EB4E2B
:106F40000F900F9094CB00D08BE594E0ADB7BEB717
:106F500012969C938E9311970E94EB4E0F900F9078
:106F600080CB0F931F93CF93DF9300D000D000D03E
:106F700087E791E0EDB7FEB7928381838091CD01E1
:106F80009091CE01A091CF01B091D00183839483E1
:106F9000A583B6830E94EB4E0F900F900F900F9039
:106FA00008EC11E1EDB7FEB7128301830E94EB4EAE
:106FB0008DB79EB740970FB6F8949EBF0FBE8DBF9A
:106FC000CDB7DEB721968FE491E0EDB7FEB792839F
:106FD0008183609125027091260280912702909111
:106FE000280220E030E041E655E40E94C6496A8369
:106FF0007B838C839D8380918B0290918C02A091E6
:107000008D02B0918E028E839F83A887B98780916D
:10701000C8029091C902A091CA02B091CB028A879E
:107020009B87AC87BD876091160270911702809193
:1070300018029091190220E030E041E655E40E94E8
:10704000C6496E877F87888B998B0E94EB4E8DB7E0
:107050009EB740960FB6F8949EBF0FBE8DBFEDB79A
:10706000FEB7128301830E94EB4E8DB79EB7409707
:107070000FB6F8949EBF0FBE8DBFCDB7DEB7219679
:1070800087E291E0EDB7FEB79283818360912D0294
:1070900070912E0280912F029091300220E030E01A
:1070A00041E655E40E94C6496A837B838C839D83B5
:1070B0008091030390910403A0910503B09106030E
:1070C0008E839F83A887B98780913502909136027D
:1070D000A0913702B09138028A879B87AC87BD8721
:1070E00060910703709108038091090390910A034E
:1070F00020E030E041E655E40E94C6496E877F8774
:10710000888B998B0E94EB4E8DB79EB740960FB639
:10711000F8949EBF0FBE8DBFEDB7FEB712830183FB
:107120000E94EB4E0F900F90DF91CF911F910F9126
:107130000895F89491E2E0E0F0E090935700849194
:10714000E2E0F0E0909357002491E4E0F0E09093C7
:107150005700E49190E0A0E0B0E0DC019927882797
:1071600030E040E050E0542F432F322F2227820F8F
:10717000931FA41FB51F8E0F911DA11DB11D8093DC
:10718000870290938802A0938902B0938A02789430
:1071900008952F923F924F925F926F927F928F92BB
:1071A0009F92AF92BF92CF92DF92EF92FF920F9396
:1071B0001F93DF93CF93CDB7DEB760970FB6F894E8
:1071C000DEBF0FBECDBF80E88093610082E0809378
:1071D00061000E9499388091870290918802A09165
:1071E0008902B0918A02853027E992072EE1A20731
:1071F00020E0B20709F435C784E690E09093E001FF
:107200008093DF010E94C71281E00E9413120E9446
:1072100071448AE294E469E574E40E94324E02C04B
:107220000E9445440E943F448823D1F70E94C9131D
:107230000E94E9228091D901882341F520914801DB
:107240003091490140914A0150914B0160E070E05A
:1072500080EA91E40E945D4926EA3BE944EC5CE364
:107260000E94154B2091690130916A0140916B0198
:1072700050916C010E945E499B01AC012093610119
:107280003093620140936301509364018091200325
:1072900081FD12C080E090E07C0108C00894E11CF0
:1072A000F11CF5E6EF16F10409F4E1C60E943E2058
:1072B0008091200381FFF2CF28EC31E18CEF90E048
:1072C0009C838B83A5EEB0E0BE83AD83EAECF0E057
:1072D000F887EF838AEA90E09A878987ABE9B0E084
:1072E000BC87AB87ECE8F0E0FE87ED87388B2F8713
:1072F00002C00E943E208091200381FFFACF80913E
:1073000020038D7F809320030E94581C0E943F44DD
:10731000882379F38091B0039091B1030E947C207F
:107320008130910509F4FAC08230910509F479C0E1
:107330008330910509F4DCC08430910509F4F7C06D
:107340008530910509F45FC2AAE02A2E3324442433
:107350005524662477248824992400D0EF85F88961
:10736000ADB7BEB71296FC93EE9311970E94EB4E09
:107370000F900F909101A201B301C4010E945A2FF6
:10738000009709F0B6CF8091D801813009F430C35D
:10739000F22DF33709F465C19101A201B301C401D3
:1073A000F3E7AF2EE3E6BE2ECC24DD24EE24FF244B
:1073B00000E010E00E946B458230E0F5322D353759
:1073C00009F472C39101A201B301C40105E7A02E23
:1073D000BB24CC24DD24EE24FF2400E010E00E9436
:1073E0006B45823008F0D4C1822D823609F435C451
:1073F0009101A201B301C40112E6A12EBB24CC2449
:10740000DD24EE24FF2400E010E00E946B45823072
:1074100008F06FC3922D913609F478C50E947F2938
:1074200068CF2090CD023324442455246624772449
:10743000430193CFF22DF93609F4E1C29101A20183
:10744000B301C401F9E6AF2EE2E7BE2ECC24DD2461
:10745000EE24FF2400E010E00E946B45823008F02B
:1074600020C1322D3D3609F4ADC49101A201B30112
:10747000C4010DE6A02E15E6B12ECC24DD24EE24A9
:10748000FF2400E010E00E946B45823008F081C3C9
:10749000922D993609F4AFC5B22DBC3609F0BECF96
:1074A000E32DE43609F0BACF442009F0B7CF5520D8
:1074B00009F0B4CF662009F0B1CF772009F0AECF44
:1074C000882009F0ABCF992009F0A8CF8091A501C1
:1074D000882309F4A3CFF1E0F093DD010E94751237
:1074E0008091A401882309F404CF0E94E94301CFCD
:1074F000F091CD02FA8319828091CE0229813A81DE
:10750000280F311DC9011901892F880F880B482EBA
:10751000582E682E782E882E982E1FCF6091B20399
:107520007091B3038AE090E00E94BF4EE2CE2091BA
:10753000CD0230E040E050E060E070E080E090E0BC
:1075400000E10E94FA44122FF32EE42ED52EC62E0F
:10755000B72EA82E292E2091CE0230E040E050E038
:1075600060E070E080E090E008E00E94FA44210FC3
:10757000F1E0211708F0F0E03F0DE1E03F1508F0E1
:10758000E0E0F30FA1E0F31708F0A0E0EA2B4E0DC6
:1075900031E04E1508F030E0E40FA1E0E41708F008
:1075A000A0E03A2B5D0DA1E05D1508F0A0E0350FDD
:1075B00041E0351708F040E0A42B6C0D51E06C154C
:1075C00008F050E0A60F41E0A61708F040E0542B69
:1075D0007B0D41E07B1508F040E0570F61E0571745
:1075E00008F060E0462B8A0D61E08A1508F060E043
:1075F000480F71E0481708F070E0672B920D960F66
:107600008091CF02820F61E0821708F060E06F0F77
:1076100071E06F1708F070E07E0F21E07E1708F030
:1076200020E0E22FE30F21E0E31708F020E0322F03
:107630003A0FF1E03A1708F0F0E0F50F21E0F51706
:1076400008F020E0240F51E0241708F050E0282E25
:10765000362E472E5E2E632E7F2E822E952E990E6D
:107660007CCE232D233609F097CE442009F094CE0A
:10767000552009F091CE662009F08ECE772009F0D2
:107680008BCE882009F088CE992009F085CE0E9403
:10769000B1378091A401882309F42BCE0E94E943DD
:1076A00028CE922D953609F474C39101A201B3013D
:1076B000C401B5E6AB2EA4E7BA2EF1E6CF2EE4E680
:1076C000DE2EEE24FF2400E010E00E946B458230A5
:1076D00008F0AEC2F22DF33709F436C4322D333739
:1076E00009F09CCE832D843709F098CE442009F010
:1076F00095CE552009F092CE662009F08FCE7720E6
:1077000009F08CCE882009F089CE992009F086CE28
:107710008091B0039091B1030E947C20803191054B
:107720000CF488C4F8948DEC92E00E94164D90936E
:10773000AF038093AE0382ED92E00E94164D8093DA
:10774000AD0385ED92E00E94164D8093AC0388ED69
:1077500092E00E94164D8093AB038BED92E00E9465
:10776000164D8093AA038EED92E00E94164D8093F1
:10777000A903789400D0EF85F889ADB7BEB712960B
:10778000FC93EE9311970E94EB4E0F900F9081CFD8
:10779000E22DE33609F47FC29101A201B301C401D5
:1077A000B3E6AB2EA3E6BA2ECC24DD24EE24FF24D0
:1077B00000E010E00E946B45823008F0BFC1222D2E
:1077C000263709F44BC3322D3D3609F027CE832DE1
:1077D000823609F023CE442009F020CE552009F04E
:1077E0001DCE662009F01ACE772009F017CE88202A
:1077F00009F014CE992009F011CEB1E0B093D80170
:107800000E94422976CD2091CD0230E040E050E048
:1078100060E070E080E090E008E10E94FA44122FFE
:10782000F32EE42ED52EC62EB72EA82E292E20916B
:10783000CE0230E040E050E060E070E080E090E0B8
:1078400000E10E94FA44210FF1E0211708F0F0E076
:107850003F0DE1E03F1508F0E0E0F30FA1E0F31782
:1078600008F0A0E0EA2B4E0D31E04E1508F030E0B4
:10787000E40FA1E0E41708F0A0E03A2B5D0D41E031
:107880005D1508F040E0350FA1E0351708F0A0E0E5
:107890004A2B6C0D51E06C1508F050E0460FA1E04A
:1078A000461708F0A0E05A2B7B0D61E07B1508F02D
:1078B00060E0570FA1E0571708F0A0E06A2B8A0D8F
:1078C00071E08A1508F070E0680FA1E0681708F011
:1078D000A0E07A2B920D970F1091D002120F81E049
:1078E000121708F080E0F82EFF0E81E0FF1608F076
:1078F00080E0E82EEE0E81E0EE1608F080E0D82E53
:10790000D30E81E0D31608F080E0C82EC40E81E0CB
:10791000C41608F080E0B82EB50E81E0B51608F068
:1079200080E0A82EA60E81E0A61608F080E0282EA2
:10793000290E2091CF0230E040E050E060E070E09E
:1079400080E090E008E00E94FA44210FE1E0211776
:1079500008F0E0E0FF2DF30F31E0FF1508F030E014
:10796000EF0FA1E0EF1708F0A0E03A2B4E0DF1E089
:107970004E1508F0F0E0340FA1E0341708F0A0E055
:10798000FA2B5D0D41E05D1508F040E0F50FA1E038
:10799000F51708F0A0E04A2B6C0D51E06C1508F0CB
:1079A00050E0460FA1E0461708F0A0E05A2B6B2DDF
:1079B000670F71E06B1508F070E0560FA1E05617E5
:1079C00008F0A0E07A2B8A0D61E08A1508F060E0EB
:1079D000780FA1E0781708F0A0E06A2B920D222E14
:1079E0003E2E432E5F2E3A01872E962E990EB5CC51
:1079F0009101A201B301C4010E946B2A7ACC232D0C
:107A0000223709F01BCD442009F018CD552009F08C
:107A100015CD662009F012CD772009F00FCD882012
:107A200009F00CCD992009F009CD00D000D0E985EE
:107A3000FA85ADB7BEB71296FC93EE93119780917D
:107A4000E5019091E60114969C938E9313970E9402
:107A5000EB4E0F900F900F900F908091B00390918C
:107A6000B1030E947C208230910584F08DEC92E07D
:107A70000E94164D9093E6018093E50185EE91E01A
:107A800064E470E042E050E00E94B04F00D0EF8527
:107A9000F889ADB7BEB71296FC93EE9311970E948A
:107AA000EB4E0F900F9025CC332009F08BCC442067
:107AB00009F088CC552009F085CC662009F082CCED
:107AC000772009F07FCC882009F07CCC992009F040
:107AD00079CC60919702709198028091990290916F
:107AE0009A020E94F1098091A401882309F401CC33
:107AF000FCCCA22DA83609F440C2B22DB43709F04F
:107B00008DCC332009F08ACC442009F087CC552055
:107B100009F084CC662009F081CC772009F07ECC76
:107B2000882009F07BCC992009F078CC0E94DB22D8
:107B30008091A401882309F4DCCBD7CC922D99360F
:107B400009F433C2B22DBC3609F068CCE32DE3361C
:107B500009F064CC442009F061CC552009F05ECCDA
:107B6000662009F05BCC772009F058CC882009F01A
:107B700055CC992009F052CC8091A501882309F4B5
:107B80004DCC1092DD018091A401882309F4B1CB82
:107B9000ACCCF22DF23609F47EC1322D343709F027
:107BA0003DCC832D8D3609F039CC442009F036CCFC
:107BB000552009F033CC662009F030CC772009F04D
:107BC0002DCC882009F02ACC992009F027CC81E01F
:107BD00090918A01911180E080938A01882309F4B1
:107BE0003DC231E03093D10186E391E000D000D076
:107BF000ED81FE81ADB7BEB71296FC93EE9311975F
:107C000014969C938E9313970E94EB4E0F900F90B7
:107C10000F900F908AE891E062E470E041E050E05C
:107C20000E94B04F8091A401882309F462CB5DCCFF
:107C3000922D903709F4F9C0F22DF43709F0EECB0C
:107C4000232D203709F0EACB342D303709F0E6CB6D
:107C5000852D8D3609F0E2CBAECF332009F0C8CBAD
:107C6000442009F0C5CB552009F0C2CB662009F0AD
:107C7000BFCB772009F0BCCB882009F0B9CB992085
:107C800009F0B6CB81E090E00E94BB0988B1A1E089
:107C90008A2788B92ECBF32DF33609F07DCD442009
:107CA00009F07ACD552009F077CD662009F074CD22
:107CB000772009F071CD882009F06ECD992009F068
:107CC0006BCD00D0ED85FE85ADB7BEB71296FC93A7
:107CD000EE9311970E94EB4EEF85F889ADB7BEB7D2
:107CE0001296FC93EE9311970E94EB4E80E090E089
:107CF000DC018093160290931702A0931802B093B0
:107D000019028093C8029093C902A093CA02B0934B
:107D1000CB0280938B0290938C02A0938D02B09340
:107D20008E028093250290932602A0932702B0939F
:107D300028028093070390930803A0930903B0934C
:107D40000A038093350290933602A0933702B093D2
:107D500038028093030390930403A0930503B09328
:107D6000060380932D0290932E02A0932F02B093CE
:107D700030028093CD019093CE01A093CF01B093B8
:107D8000D0018091A4010F900F90882309F4B1CA0B
:107D9000ACCBA32DA43709F088CCB42DB13609F0B3
:107DA00084CCE52DE43609F080CC662009F07DCC4A
:107DB000772009F07ACC882009F077CC992009F453
:107DC000B5CE73CC832D853609F04FCB442009F016
:107DD0004CCB552009F049CB662009F046CB7720E3
:107DE00009F043CB882009F040CB992009F03DCB26
:107DF00081E09091A501911180E08093A5018823F5
:107E000009F429C186E391E000D000D02B813C81A8
:107E1000EDB7FEB732832183948383830E94EB4EB8
:107E20000F900F900F900F9064CAA32DAC3609F0FD
:107E300003CFB42DB53609F0FFCEE52DE83609F0B5
:107E4000FBCE662009F0F8CE772009F0F5CE882029
:107E500009F0F2CE992009F4A5C0EECE332009F046
:107E6000B2CC442009F0AFCC552009F0ACCC662050
:107E700009F0A9CC772009F0A6CC882009F0A3CC82
:107E8000992009F0A0CC0E94E9228091A4018823C6
:107E900009F42FCA2ACB232D2D3609F07ECE44209B
:107EA00009F07BCE552009F078CE662009F075CE1A
:107EB000772009F072CE882009F06FCE992009F062
:107EC0006CCE81E090918B01911180E080938B01C9
:107ED000882309F4BDC086E391E000D000D0EF8193
:107EE000F885ADB7BEB71296FC93EE931197149632
:107EF0009C938E9313970E94EB4E0F900F900F90D0
:107F00000F908BE891E063E470E088CE332009F0B5
:107F100085CA442009F082CA552009F07FCA66202C
:107F200009F07CCA772009F079CA882009F076CA5E
:107F3000992009F073CA80E090E00E94BB0988B1E3
:107F400092E0892788B9D5C9232D223709F0C6CBFD
:107F5000442009F0C3CB552009F0C0CB662009F0BE
:107F6000BDCB772009F0BACB882009F0B7CB992098
:107F700009F0B4CB0E94F320BCC9332009F0BDCD79
:107F8000442009F0BACD552009F0B7CD662009F09C
:107F9000B4CD772009F0B1CD882009F0AECD99207D
:107FA00009F0ABCD0E949229A4C9A32DA33609F0F4
:107FB000C9CD442009F0C6CD552009F0C3CD6620B7
:107FC00009F0C0CD772009F0BDCD882009F0BACDE9
:107FD000992009F0B7CD8091A501882309F41ECA24
:107FE0001092DE0180918A01882309F452CB21E0AE
:107FF0002093D1014ECBA32DA43609F04DCA4420C5
:1080000009F04ACA552009F047CA662009F044CA57
:10801000772009F041CA882009F03ECA992009F06A
:108020003BCA8091A501882309F4F8C931E0309357
:10803000DE012FCB00D0EB85FC85ADB7BEB7129625
:10804000FC93EE9311970E94EB4E0F900F9021CB73
:1080500089E391E042CF89E391E0D6CE89E391E0D4
:10806000C5CD8091C40188608093C401C5C880E0FB
:1080700090E00E94BB0920C989B1807408955E9A7E
:10808000569A08955E98569808955E98569A8DED82
:1080900090E08115910511F00197F1F72FB7F89451
:1080A00056988EE190E08115910511F00197F1F756
:1080B00089B12FBF7894EEEBF0E0E115F10511F0F6
:1080C0003197F1F74E9902C081E0089580740895C8
:1080D0009FB7F894569AE0E0F0E0E115F10511F051
:1080E0003197F1F781115698E5E0F0E0E115F105DF
:1080F00011F03197F1F74E9B80E0E4E1F0E0E115FB
:10810000F10511F03197F1F756989FBFEDE0F0E0DF
:10811000E115F10511F03197F1F708950F931F93D1
:10812000182F08E0812F81700E94684016958111F8
:1081300010680150B9F7812F1F910F9108958FEFAB
:108140000E948E400895DF92EF92FF920F931F934B
:10815000CF93DF93182FEB010E944540882359F0FD
:10816000DD24DA948D2DDF91CF911F910F91FF9037
:10817000EF90DF90089580EF0E948E40DD2400E4B0
:1081800098EFE92EE00E0BC0FF2061F580E00E9421
:10819000684088818695888301500E15F9F081E04A
:1081A0000E946840F82E81E00E946840882361F7B1
:1081B000FF2051F4011728F0888180FFE7CF1017C6
:1081C00029F3D02EFF24F3948F2D0E9468408881DC
:1081D00086958068888301500E1509F7002311F2F7
:1081E0002196CECF8EEFD82EBDCF0F931F93CF9376
:1081F000DF93182FEB010E944540209789F085E519
:108200000E948E4008E089910E948E400150D9F76B
:10821000812F0E948E40DF91CF911F910F91089581
:108220008CEC0E948E40812F0E948E40DF91CF9176
:108230001F910F910895DC01CB0181159105A105D6
:10824000B10529F081509040A040B040D9F7089581
:108250000F931F93CF93DF93FB01E801608170E0E0
:10826000B181A0E06A2B7B2B803129F177FD34C0EE
:10827000DA011C92883289F0CB01929582958F7039
:1082800089279F708927F90180836F70688380E058
:10829000DF91CF911F910F910895848190E0AC01FF
:1082A000407650704036510539F386FD1CC085FD7F
:1082B0001CC0687FE1CFDB01AE7FAA0FBB1FAA0FF6
:1082C000BB1FAA0FBB1F96816CE070E0691B710990
:1082D0006A0F7B1F77FFCCCF91E0DA019C937095FA
:1082E00061957F4FC7CF6E7FC7CF6C7FC5CF0F9390
:1082F0001F93CF93DF938C01EB01FC018081BE01C2
:108300000E94A340F8018083982F91509D3F28F44C
:108310009881983211F0903191F7DF91CF911F91B0
:108320000F9108951F93CF93DF93EC010E94454076
:1083300084EBBE010E94F54081E00E946840182F46
:108340000E94454081E0112309F480E0DF91CF9144
:108350001F9108951F93CF93DF93182FEB010E9475
:1083600045400E943C40882329F482E0DF91CF9170
:108370001F91089584E4BE010E94F540113039F048
:108380000E943F4080E0DF91CF911F91089580E0EF
:10839000DF91CF911F9108954F925F926F927F92DC
:1083A0008F929F92AF92BF92CF92DF92EF92FF9205
:1083B0000F931F93DF93CF93CDB7DEB729970FB6F7
:1083C000F894DEBF0FBECDBF5C013B012A0149011D
:1083D0000E9445408EEBB5010E94F5408E010F5F73
:1083E0001F4F78017AE0C72ED12CCC0EDD1E0E94E3
:1083F0009F40F70181937F01EC15FD05C1F7C8018E
:1084000069E070E00E9445438823C1F083E029962B
:108410000FB6F894DEBF0FBECDBFCF91DF911F9195
:108420000F91FF90EF90DF90CF90BF90AF909F9013
:108430008F907F906F905F904F900895F5018081AD
:10844000B801A301920184010E94284180E0DFCF9E
:108450005F926F927F928F929F92AF92BF92CF92D4
:10846000DF92EF92FF920F931F93DF93CF93CDB7DD
:10847000DEB729970FB6F894DEBF0FBECDBF582EDA
:108480004B013A0159018EEB60E070E00E94F5402B
:108490008E010F5F1F4F7801EAE0CE2ED12CCC0E5B
:1084A000DD1E0E949F40F70181937F01EC15FD05C1
:1084B000C1F7C80169E070E00E9445438823B9F024
:1084C00083E029960FB6F894DEBF0FBECDBFCF91E3
:1084D000DF911F910F91FF90EF90DF90CF90BF90B1
:1084E000AF909F908F907F906F905F900895852DB3
:1084F000B801A401930185010E94284180E0E1CFE9
:10850000EF92FF920F931F93DF93CF93CDB7DEB718
:1085100028970FB6F894DEBF0FBECDBF182F062FD9
:108520007E010894E11CF11CC701A4EBB1E038E026
:108530000D90FC010192CF013150D1F7242F332748
:1085400027FD309541E752E0249FC001259F900D03
:10855000349F900D112464E670E00E94984BAB01AB
:1085600064E6069FB0011124460F571FF701CE01A4
:108570000996619170E026173707B1F0E817F907FF
:10858000C1F7112319F0509541955F4FCA01289604
:108590000FB6F894DEBF0FBECDBFCF91DF911F9114
:1085A0000F91FF90EF9008954F5F5F4FEACF0F93C9
:1085B0001F93DF93CF93CDB7DEB72B970FB6F89409
:1085C000DEBF0FBECDBF182F092F885F612F792F17
:1085D0000E94AA41882371F064E371E2CB012B96DB
:1085E0000FB6F894DEBF0FBECDBFCF91DF911F91C4
:1085F0000F9108956AE673E883E090E00E941B41C2
:10860000812F902FBE016F5F7F4FAE014E5F5F4F96
:108610009E012D5F3F4F0E94CC418823E9F69E01C9
:108620002C5F3F4FD901ECEAF1E088E001900D9218
:108630008150E1F74B81E42FF0E061E772E0E69FC3
:10864000C001E79F900DF69F900D112464E670E045
:108650000E94984B9A8184E6989FC0011124680F6C
:10866000791FF901CE010C962191421759F0E817B4
:10867000F907D1F78981882309F4B0CF7095619506
:108680007F4FACCF6F5F7F4FF5CF61157105E1F084
:10869000E82FF92F20E030E080E0A8E1419198E058
:1086A00004C08695915051F04695542F582750FF9D
:1086B000F8CF8A27869580689150B1F72F5F3F4F9A
:1086C0006217730759F7089580E008951F920F927B
:1086D0000FB60F920BB60F9211248F93EF93FF9367
:1086E0008091C600E0912503F0E0EF73F070EA5D41
:1086F000FC4F8083809125038F5F80932503FF913A
:10870000EF918F910F900BBE0F900FBE0F901F90A7
:1087100018951F920F920FB60F920BB60F9211245D
:108720008F939F93EF93FF939091660380916803DB
:108730009817D1F0E0916803F0E0EF73F070E7591B
:10874000FC4F80818093C600809168038F5F809387
:108750006803FF91EF919F918F910F900BBE0F9047
:108760000FBE0F901F9018958091C1008F7D809350
:10877000C100EFCF161617061CF5DC0120E030E033
:1087800090912503809167039817D1F3E0916703D7
:10879000F0E0EF73F070EA5DFC4F40818091670379
:1087A0008F5F809367034D93CD014D3029F02F5F8C
:1087B0003F4F2617370724F3FC011082C9010895A3
:1087C00020E030E0F9CF8091660390916803891B27
:1087D000089540E450E09091660320916803921B55
:1087E0009A01291B310923303105ACF3E09166036E
:1087F000F0E0EF73F070E759FC4F808380916603DF
:108800008F5F809366038091C10080628093C10076
:108810000895CF93DF93EC01FC018491882341F00C
:1088200021960E94E943FE01219684918823C9F78D
:10883000DF91CF910895CF93DF93EC018881882356
:1088400031F021960E94E94389918823D9F7DF917D
:10885000CF9108951F93182F8A3039F0812F0E94ED
:10886000E94380E090E01F9108958DE00E94E94384
:10887000812F0E94E94380E090E01F91089580914C
:10888000250390916703891B08959091250380919A
:1088900067039817D1F3E0916703F0E0EF73F0708E
:1088A000EA5DFC4F8081909167039F5F909367031F
:1088B000089590912503809167039817D1F3E09173
:1088C0006703F0E0EF73F070EA5DFC4F80819091F8
:1088D00067039F5F9093670390E008950E94E943C8
:1088E000089585E090E09093C5008093C40082E0F5
:1088F0008093C0008AE98093C10008958091A90304
:108900008F5F8093A9038C3309F008951092A90317
:108910008091AA038F5F8093AA038C33B1F71092E2
:10892000AA038091AB038F5F8093AB03883169F713
:108930001092AB038091AC038F5F8093AC038032C5
:10894000B9F08F31F1F08E3169F18D31B1F1809153
:10895000AD038D30D1F681E08093AD038091AE03FD
:108960009091AF0301969093AF038093AE03089567
:108970008091AD038F5F8093AD0391E09093AC0342
:10898000E8CF8091AD03843031F0863021F089301A
:1089900011F08B30F1F68F5F8093AD0391E09093EF
:1089A000AC03D7CF8091AD03823099F683E08093FA
:1089B000AD0381E08093AC0308958091AD038230D4
:1089C00041F64091AE03E091AF03842F9E2F64E601
:1089D00070E00E94844B009751F4842F9E2F60E931
:1089E00071E00E94844B882309F48FCFDFCF842F5E
:1089F0008370F9CF0F93DF93CF93CDB7DEB7609736
:108A00000FB6F894DEBF0FBECDBF002309F459C0E6
:108A100029833A834B835C836D837E838F8398871E
:108A2000E0E2E01B29813A814B815C811E16BCF09B
:108A300019861A861B861C868E2F992787FD90958E
:108A4000909581959F4F04C0220F331F441F551FDF
:108A50008A95D2F72D873E874F87588B2AC0CA0147
:108A6000B901002E04C0660F771F881F991F0A9452
:108A7000D2F769877A878B879C87DA01C90104C09E
:108A8000B695A79597958795EA95D2F72D813E8162
:108A90004F81588504C0220F331F441F551F0A956C
:108AA000D2F7822B932BA42BB52B8D879E87AF8774
:108AB000B88B29853A854B855C856D857E858F854C
:108AC000988960960FB6F894DEBF0FBECDBFCF91E8
:108AD000DF910F910895A0E1B0E0E1E7F5E40C9497
:108AE000D54B29833A834B835C836D837E838F834D
:108AF0009887A986BA86CB86DC86ED86FE860F87A8
:108B0000188B2D813E814F8158858D859E85AF853F
:108B1000B889281739074A075B07C8F082179307F7
:108B2000A407B50790F029813A814B815C81898542
:108B30009A85AB85BC85281739074A075B0738F04B
:108B400082179307A407B50720F482E003C080E0F2
:108B500001C081E06096EAE00C94F14B2F923F92C5
:108B60004F925F926F927F928F929F92AF92BF923D
:108B7000CF92DF92EF92FF920F931F93DF93CF93E9
:108B8000CDB7DEB763970FB6F894DEBF0FBECDBF8B
:108B90006C017F876E87FC0117821682838181FDBD
:108BA00004C06FC34C855D8504C01E010894211C60
:108BB000311CF6019381EE85FF8593FD859193FF2E
:108BC0008191FF87EE87882309F457C3853241F4EA
:108BD00093FD859193FF8191FF87EE87853259F44C
:108BE00090E0B6014A8B5B8B0E94BF4E4A895B893D
:108BF0005D874C87D7CF10E0FF2400E00032B0F44F
:108C00008B3269F08C3228F4803251F0833271F467
:108C10000BC08D3239F0803349F401602CC0026002
:108C2000046029C0086027C0006125C007FD2EC070
:108C3000282F20532A3098F406FF08C0812F880F70
:108C4000182F110F110F180F120F15C08F2D880F2D
:108C5000F82EFF0CFF0CF80EF20E00620CC08E32E4
:108C600021F406FD0AC3006406C08C3611F40068C6
:108C700002C0883659F4EE85FF8593FD859193FFF8
:108C80008191FF87EE87882309F0B8CF982F9554FC
:108C9000933018F40061805E06C0982F955693308B
:108CA00008F09BC10F7E06FF16E06FE3E62EE02280
:108CB000853619F4F0E4EF2A07C0863619F420E867
:108CC000E22A02C011111150E7FE06C01C3340F425
:108CD000912E939427E00BC0183030F4212F06C05A
:108CE00027E03CE3932E03C027E017E09924CA0154
:108CF00004969D878C87FA016081718182819381BE
:108D0000A101092D0E94344D5C016980262D30E0BF
:108D1000398B288B60FE03C0388933FF06C0E1FC25
:108D200006C0E2FE06C000E205C00DE203C00BE291
:108D300001C000E0888999898C7090700097C1F11A
:108D4000002311F084E001C083E08F1558F4F81A75
:108D5000E3FC09C080E290E0B6010E94BF4EFA94A5
:108D6000C9F701C0FF24002329F0802F90E0B6014D
:108D70000E94BF4E888983FD03C00EEC11E10EC036
:108D80000AEC11E10BC0A114B10409F0805290E08B
:108D9000B6010E94BF4E0F5F1F4F05C0AE2CBB2413
:108DA00090E1A922BB24F8018491882361F762C273
:108DB000E7FE0EC09A0CF889F4FF04C08A81813363
:108DC00009F49A94191454F5292D293050F52DC021
:108DD000E6FC2BC0812F90E08A159B054CF03CEF00
:108DE000A3163FEFB30624F080E8E82A01C0115033
:108DF000112349F0E2E0F0E0EC0FFD1FE10FF11D5F
:108E000080818033A1F3E7FE10C0912E9394812FCF
:108E100090E0A816B90644F41A1907C0992493944F
:108E200004C098E0992E01C010E0E7FE07C01A14B4
:108E30001B043CF495012F5F3F4F05C025E030E057
:108E400002C021E030E0002311F02F5F3F4F1123DB
:108E500029F0812F90E00196280F391F8F2D90E087
:108E60002817390714F4F21A01C0FF244E2C552498
:108E7000C20189709070009749F406C080E290E0CA
:108E8000B6010E94BF4EFA94FF20C1F7002329F0DB
:108E9000802F90E0B6010E94BF4E43FC09C006C07F
:108EA00080E390E0B6010E94BF4EFA94FF20C1F724
:108EB000E7FE46C03501B7FE02C0662477242501CF
:108EC0000894411C511C46185708420C531CF501CC
:108ED000E919F1094F01812F90E000271127081BA4
:108EE000190BFFEF6F16FFEF7F0629F48EE290E07B
:108EF000B6010E94BF4EA614B70434F0861497043E
:108F00001CF4F201808101C080E3089461087108BB
:108F10000894411C511C601671062CF090E0B601BB
:108F20000E94BF4EDECF6A147B0441F49A819633CF
:108F300020F4953319F4F889F4FF81E390E049C0F7
:108F40008A81813311F02FEE622290E0B6010E94F7
:108F5000BF4E112389F08EE290E0B6010E94BF4E11
:108F600002E0F101E00FF11D0F5F808190E0B6019A
:108F70000E94BF4E1150A9F744FE03C085E490E063
:108F800002C085E690E0B6010E94BF4EB7FC05C066
:108F9000A114B10441F464FE06C0B094A194B108D8
:108FA000B3948DE201C08BE290E0B6010E94BF4E07
:108FB00080E305C08F5FE6EFFFEFAE0EBF1EFAE065
:108FC000AF16B104BCF790E0B6010E94BF4EC501D8
:108FD000C096B6010E94BF4E4DC1833631F0833733
:108FE00089F0833509F059C022C09A012E5F3F4FA6
:108FF0003D872C87FA0180818983310181E0A82E89
:10900000B12C13C09A012E5F3F4F3D872C87FA0188
:109010006080718006FF03C0612F70E002C06FEFB7
:109020007FEFC3010E941F4E5C010F7714C09A01AD
:109030002E5F3F4F3D872C87FA016080718006FFCD
:1090400003C0612F70E002C06FEF7FEFC3010E9489
:10905000144E5C01006803FD1CC006C080E290E075
:10906000B6010E94BF4EFA948F2D90E0A816B90663
:10907000A8F30FC0F30107FD859107FF81913F0120
:1090800090E0B6010E94BF4EF110FA940894A10836
:10909000B108A114B10471F7EDC0843611F089361E
:1090A00061F507FF0BC09A012C5F3F4F3D872C876E
:1090B000FA0160817181828193810CC09A012E5FD7
:1090C0003F4F3D872C87FA0160817181882777FDAA
:1090D0008095982F0F7697FF08C090958095709592
:1090E00061957F4F8F4F9F4F0068A1012AE030E0CC
:1090F0000E94424F982E921841C0853721F40F7E6E
:109100002AE030E020C0097F8F36A9F0803720F4B4
:10911000883509F0B2C00BC0803721F0883709F0DC
:10912000ACC001C0006104FF09C0046007C004FFB7
:1091300008C0066006C028E030E005C020E130E04D
:1091400002C020E132E007FF0AC0CA0104969D87F1
:109150008C87FA01608171818281938109C0CA0183
:1091600002969D878C87FA016081718180E090E092
:10917000A1010E94424F982E92180F7706FF09C056
:109180000E7F911630F404FF06C002FD04C00F7E6E
:1091900002C0E92C01C0E12E802F90E004FF0CC03A
:1091A000FE01E90DF11D2081203311F4097E09C073
:1091B000E39402FF06C004C086789070009709F01F
:1091C000E394A02EBB2403FD14C000FF0FC0EF14D6
:1091D00028F4192D1F0D1E19EF2C08C0192D06C0DB
:1091E00080E290E0B6010E94BF4EE394EF14C0F31A
:1091F00004C0EF1410F4FE1801C0FF24A4FE0FC039
:1092000080E390E0B6010E94BF4EA2FE1FC0A1FE07
:1092100003C088E590E010C088E790E00DC0C5016C
:1092200086789070009791F0A1FC02C080E201C0A6
:109230008BE207FD8DE290E0B6010E94BF4E06C0B2
:1092400080E390E0B6010E94BF4E11509116C0F32A
:109250009A94F101E90DF11D808190E0B6010E9420
:10926000BF4E9920A9F706C080E290E0B6010E94A7
:10927000BF4EFA94FF20C1F795CCF60126813781C5
:1092800002C02FEF3FEFC90163960FB6F894DEBF1F
:109290000FBECDBFCF91DF911F910F91FF90EF9047
:1092A000DF90CF90BF90AF909F908F907F906F9006
:1092B0005F904F903F902F9008955058BB27AA275A
:1092C0000ED075C166D130F06BD120F031F49F3FE4
:1092D00011F41EF45BC10EF4E095E7FB51C1E92FD8
:1092E00077D180F3BA17620773078407950718F0E0
:1092F00071F49EF58FC10EF4E0950B2EBA2FA02DC0
:109300000B01B90190010C01CA01A0011124FF2732
:10931000591B99F0593F50F4503E68F11A16F0402D
:10932000A22F232F342F4427585FF3CF469537952C
:109330002795A795F0405395C9F77EF41F16BA0BF1
:10934000620B730B840BBAF09150A1F0FF0FBB1F9F
:10935000661F771F881FC2F70EC0BA0F621F731FE8
:10936000841F48F4879577956795B795F7959E3F45
:1093700008F0B3CF9395880F08F09927EE0F9795D3
:1093800087950895D9D008F481E008950CD00FC1D5
:1093900007D140F0FED030F021F45F3F19F0F0C06B
:1093A000511139C1F3C014D198F39923C9F355234E
:1093B000B1F3951B550BBB27AA27621773078407C8
:1093C00038F09F5F5F4F220F331F441FAA1FA9F37E
:1093D00033D00E2E3AF0E0E830D091505040E69570
:1093E000001CCAF729D0FE2F27D0660F771F881FD1
:1093F000BB1F261737074807AB07B0E809F0BB0BC0
:10940000802DBF01FF2793585F4F2AF09E3F5105E3
:1094100068F0B6C000C15F3FECF3983EDCF3869580
:1094200077956795B795F7959F5FC9F7880F911D59
:109430009695879597F90895E1E0660F771F881F45
:10944000BB1F621773078407BA0720F0621B730BF8
:10945000840BBA0BEE1F88F7E095089504D068944A
:10946000B111D9C00895BCD088F09F5790F0B92FA2
:109470009927B751A0F0D1F0660F771F881F991F69
:109480001AF0BA95C9F712C0B13081F0C3D0B1E07B
:109490000895C0C0672F782F8827B85F39F0B93F8B
:1094A000CCF3869577956795B395D9F73EF490956B
:1094B0008095709561957F4F8F4F9F4F0895E894E9
:1094C00009C097FB3EF490958095709561957F4F0C
:1094D0008F4F9F4F9923A9F0F92F96E9BB279395BA
:1094E000F695879577956795B795F111F8CFFAF4CA
:1094F000BB0F11F460FF1BC06F5F7F4F8F4F9F4FFB
:1095000016C0882311F096E911C0772321F09EE858
:10951000872F762F05C0662371F096E8862F70E0BE
:1095200060E02AF09A95660F771F881FDAF7880F98
:109530009695879597F90895990F0008550FAA0BEE
:10954000E0E8FEEF16161706E807F907C0F0121656
:109550001306E407F50798F0621B730B840B950B59
:1095600039F40A2661F0232B242B252B21F40895AE
:109570000A2609F4A140A6958FEF811D811D08954B
:1095800097F99F6780E870E060E008959FEF80ECB6
:10959000089500240A941616170618060906089559
:1095A00000240A9412161306140605060895092EBF
:1095B0000394000C11F4882352F0BB0F40F4BF2B2E
:1095C00011F460FF04C06F5F7F4F8F4F9F4F08956E
:1095D00057FD9058440F551F59F05F3F71F0479564
:1095E000880F97FB991F61F09F3F79F08795089549
:1095F000121613061406551FF2CF4695F1DF08C068
:10960000161617061806991FF1CF86957105610584
:1096100008940895E894BB2766277727CB0197F92C
:1096200008958ADF08F48FEF08950BD0C0CFB1DF23
:1096300028F0B6DF18F0952309F0A2CFA7CF1124A8
:10964000EACFC6DFA0F3959FD1F3950F50E0551FE9
:10965000629FF001729FBB27F00DB11D639FAA2787
:10966000F00DB11DAA1F649F6627B00DA11D661FD6
:10967000829F2227B00DA11D621F739FB00DA11DF7
:10968000621F839FA00D611D221F749F3327A00DB1
:10969000611D231F849F600D211D822F762F6A2F4D
:1096A00011249F5750408AF0E1F088234AF0EE0FD2
:1096B000FF1FBB1F661F771F881F91505040A9F7DF
:1096C0009E3F510570F05CCFA6CF5F3FECF3983E14
:1096D000DCF3869577956795B795F795E7959F5F46
:1096E000C1F7FE2B880F911D9695879597F90895E0
:1096F000991B79E004C0991F961708F0961B881FE4
:109700007A95C9F780950895AA1BBB1B51E107C044
:10971000AA1FBB1FA617B70710F0A61BB70B881F01
:10972000991F5A95A9F780959095BC01CD01089590
:1097300097FB092E07260AD077FD04D0E5DF06D077
:1097400000201AF4709561957F4F0895F6F7909573
:1097500081959F4F0895A1E21A2EAA1BBB1BFD0104
:109760000DC0AA1FBB1FEE1FFF1FA217B307E40700
:10977000F50720F0A21BB30BE40BF50B661F771F58
:10978000881F991F1A9469F7609570958095909538
:109790009B01AC01BD01CF0108952F923F924F92E2
:1097A0005F926F927F928F929F92AF92BF92CF9271
:1097B000DF92EF92FF920F931F93CF93DF93CDB77A
:1097C000DEB7CA1BDB0B0FB6F894DEBF0FBECDBFF2
:1097D00009942A88398848885F846E847D848C84C3
:1097E0009B84AA84B984C884DF80EE80FD800C81CC
:1097F0001B81AA81B981CE0FD11D0FB6F894DEBFAF
:109800000FBECDBFED0108952F923F924F925F9210
:109810006F927F929F92AF92BF92CF92DF92EF9220
:10982000FF920F931F93CF93DF933B01EA016115E2
:10983000710519F0FB0180839183209739F09E0117
:10984000225030402332310508F0D5C0C82ED92E21
:10985000F60111916F017F01812F90E00E940C4E63
:109860000097B1F71D3231F4F60111917F0199246F
:10987000939406C01B3219F4F60111917F019924CB
:10988000209719F0C031D105D1F4103389F4F701D4
:109890008081883711F0883559F4F701118182E011
:1098A00090E0E80EF91E92E0992AC0E1D0E007C0EE
:1098B000209729F41033B1F0CAE0D0E02BC0CA30B1
:1098C000D10541F1C031D10521F0C830D105A9F44D
:1098D00009C02FEFA22E2FEFB22E2FEFC22E2FE0B6
:1098E000D22E20C0C8E0D0E09FEFA92E9FEFB92E66
:1098F0009FEFC92E9FE1D92E15C09E01442737FD49
:109900004095542F6FEF7FEFCB010E94AB4B590175
:109910006A0108C089E9A82E89E9B82E89E9C82E0C
:1099200089E1D82E60E020E030E0A9011E01442446
:1099300037FC4094542C012F00530A3060F0812FE3
:1099400081548A3110F4075006C0812F81568A3124
:1099500050F5012F0755802F90E08C179D071CF5BF
:109960006F3FE9F0A216B306C406D506A8F0CA01F7
:10997000B901A20191010E94D0529B01AC01802F3C
:1099800090E0A0E0B0E0280F391F4A1F5B1F2817A6
:1099900039074A075B0710F46FEF01C061E0F70178
:1099A00011917F01C8CF6114710481F0662339F0F1
:1099B0000894E108F108F301F182E08207C091FE0A
:1099C00005C0C7010297F3019183808390FE07C011
:1099D00050954095309521953F4F4F4F5F4F67FF12
:1099E0000DC082E290E09093B7038093B6032FEF0F
:1099F0003FEFA90103C020E030E0A901B901CA018D
:109A0000DF91CF911F910F91FF90EF90DF90CF905A
:109A1000BF90AF909F907F906F905F904F903F90DE
:109A20002F900895662777270C942051FC018827F2
:109A30009927E89421912032E9F3293010F02E3053
:109A4000C8F32B3241F02D3239F4689404C00E94DF
:109A50002A4E820F911D219120532A30C0F31EF40B
:109A6000909581959F4F0895283008F027E033277F
:109A7000DA01990F311D87FD91600096610571052E
:109A800039F432602E5F3D9330E32A95E1F7089573
:109A90009F3F30F080387105610509F03C5F3C5F05
:109AA0003D93913008F08068911DDF93CF931F9311
:109AB0000F93FF92EF92192F987F9695E92F969525
:109AC0009695E90FFF27E45DFD4E99273327EE2495
:109AD000FF24A701E70105900894079428F4360FA6
:109AE000E71EF81E491F511D660F771F881F991F1B
:109AF0000694A1F70590079428F4E70EF81E491F75
:109B0000561FC11D770F881F991F661F0694A1F766
:109B10000590079428F4F80E491F561FC71FD11D42
:109B2000880F991F661F771F0694A1F70590079469
:109B300020F4490F561FC71FD81F990F661F771FA4
:109B4000881F0694A9F784911095177041F0D69557
:109B5000C79557954795F794E7941A95C1F7E2EDA5
:109B6000F1E1689415901591359165919591059065
:109B70007FE27395E118F10A430B560BC90BD0092C
:109B8000C0F7E10CF11E431F561FC91FD01D7EF404
:109B9000703311F48A95E6CFE894015030F0080F45
:109BA0000AF40027021708F4202F2395022F7A3396
:109BB00028F079E37D932A95E9F710C07D932A95E3
:109BC00089F6069497956795379517951794E11838
:109BD000F10A430B560BC90BD00998F023957E91DF
:109BE00073957A3308F070E37C932013B8F77E9175
:109BF00070617D9330F0839571E37D9370E32A95D6
:109C0000E1F71124EF90FF900F911F91CF91DF9119
:109C1000992787FD909508959111A0C4803219F07D
:109C200089508550D0F70895FC010590615070402F
:109C30000110D8F7809590958E0F9F1F0895FC0115
:109C40006150704001900110D8F7809590958E0F6B
:109C50009F1F08957AE0979F902D879F802D910DEB
:109C6000112408950F931F93CF93DF938C01EB0181
:109C7000009711F42097C9F181E090E06EE070E068
:109C80000E94C84FFC019C01009789F180E8838302
:109C9000209771F0D387C28781E883838091B003D6
:109CA0009091B103009721F4F093B103E093B003D6
:109CB00001151105E1F0118700878381826083839C
:109CC0008091B2039091B303009789F4F093B303AA
:109CD000E093B2038091B4039091B503009739F4F7
:109CE000F093B503E093B40302C020E030E0C90173
:109CF000DF91CF911F910F910895CF93DF93EC01E6
:109D00003B8130FF36C036FF09C03F7B3B838E81ED
:109D10009F8101969F838E832A8129C032FF0FC0C5
:109D2000E881F9818081992787FD9095009719F442
:109D300030623B831EC03196F983E88311C0EA8507
:109D4000FB85CE01099597FF0BC02B813FEF8F3F1D
:109D5000930711F480E101C080E2822B8B8309C05C
:109D60002E813F812F5F3F4F3F832E83282F30E08E
:109D700002C02FEF3FEFC901DF91CF9108950F93FC
:109D80001F93CF93DF938C01EB018B8181FF1BC06D
:109D900082FF0DC02E813F818C819D81281739075C
:109DA00064F4E881F9810193F983E88306C0E885CA
:109DB000F985802F0995009731F48E819F81019656
:109DC0009F838E8302C00FEF1FEFC801DF91CF91F9
:109DD0001F910F910895DF93CF93CDB7DEB7FE01AA
:109DE0003596619171918091B2039091B303DC013A
:109DF00013962C911397286013962C93AF010E9411
:109E0000AE45E091B203F091B3032381277F238312
:109E1000CF91DF910895EF92FF920F931F93CF930D
:109E2000DF938C01E091B203F091B303838181FF52
:109E30001FC0C0E0D0E00AC0DB011896ED91FC9194
:109E400019970995009711F0CFEFDFEFF801819195
:109E50008F016091B2037091B303882369F7DB012E
:109E60001896ED91FC9119978AE00995009711F0E9
:109E7000CFEFDFEFCE01DF91CF911F910F91FF90D8
:109E8000EF900895FA01AA27283051F1203181F18D
:109E9000E8946F936E7F6E5F7F4F8F4F9F4FAF4FF2
:109EA000B1E03ED0B4E03CD0670F781F891F9A1F05
:109EB000A11D680F791F8A1F911DA11D6A0F711DB9
:109EC000811D911DA11D20D009F468943F912AE0C5
:109ED000269F11243019305D3193DEF6CF010895AD
:109EE000462F4770405D4193B3E00FD0C9F7F6CFDE
:109EF000462F4F70405D4A3318F0495D31FD4052A6
:109F0000419302D0A9F7EACFB4E0A695979587953B
:109F100077956795BA95C9F700976105710508951A
:109F20009B01AC010A2E06945795479537952795C6
:109F3000BA95C9F7620F731F841F951FA01D08955E
:109F4000DC01CB01FC01F999FECF06C0F2BDE1BDF9
:109F5000F89A319600B40D9241505040B8F70895E8
:109F6000DC01CB0103C02D910E94BB4F41505040FA
:109F7000D0F70895262FF999FECF1FBA92BD81BD63
:109F800020BD0FB6F894FA9AF99A0FBE019608957B
:109F9000EF92FF920F931F93CF93DF93689F8001FF
:109FA000699F100D789F100D1124C8010E94ED4F7C
:109FB000E82EE7017E01F92EE701209731F08E2D82
:109FC00060E070E0A8010E94C952CE01DF91CF91FC
:109FD0001F910F91FF90EF900895CF93DF93823000
:109FE000910510F482E090E0E091BA03F091BB0398
:109FF00040E050E020E030E026C0608171816817C9
:10A000007907E0F06817790781F48281938121153F
:10A01000310531F0D90113969C938E9312972BC082
:10A020009093BB038093BA0326C04115510519F0E4
:10A030006417750718F4AB01E901DF019F01728114
:10A040006381E72FF62F3097C1F64115510501F1D5
:10A05000481B590B4430510580F412968D919C9108
:10A060001397209719F09B838A8304C09093BB03B6
:10A070008093BA03FD01329646C0FD01E40FF51F3F
:10A08000819391934250504011965C934E933BC004
:10A090002091B8033091B9032115310541F4209185
:10A0A000BE013091BF013093B9032093B8032091D2
:10A0B000C0013091C1012115310541F42DB73EB7E2
:10A0C0004091BC015091BD01241B350BE091B803B8
:10A0D000F091B903E217F307A0F42E1B3F0B2817EA
:10A0E000390778F0AC014E5F5F4F2417350748F011
:10A0F0004E0F5F1F5093B9034093B8038193919320
:10A1000002C0E0E0F0E0CF01DF91CF910895CF935E
:10A11000DF93009709F491C0FC01329713821282F9
:10A120006091BA037091BB036115710581F42081C0
:10A130003181280F391F8091B8039091B90382179C
:10A14000930799F5F093B903E093B80376C0DB0168
:10A1500080E090E002C0CD01D901AE17BF0748F4FE
:10A1600012962D913C91139721153105A1F7CD0140
:10A1700021C0B383A283EF01499159919E01240F1D
:10A18000351FA217B30779F42D913C911197240F35
:10A19000351F2E5F3F4F3183208312962D913C91C6
:10A1A000139733832283009729F4F093BB03E09342
:10A1B000BA0343C0DC011396FC93EE9312974D91C2
:10A1C0005D91A40FB51FEA17FB0769F42081318167
:10A1D000240F351F2E5F3F4FEC01398328832281E6
:10A1E00033813B832A83E0E0F0E002C0FB01BC0145
:10A1F000DB0112968D919C9113970097B9F79B0103
:10A200002E5F3F4F8D919C911197820F931F40912C
:10A21000B8035091B9034817590779F4309729F4D6
:10A220001092BB031092BA0302C013821282225012
:10A2300030403093B9032093B803DF91CF91089554
:10A240006F927F928F929F92AF92BF92CF92DF9246
:10A25000EF92FF920F931F93DF93CF930F92CDB79F
:10A26000DEB75B016115710521F0DB018C9311965E
:10A270009C93482F592F6A01F601E1906F018F01DD
:10A280008E2D90E00E940C4E0097B1F7FE2DFD320E
:10A2900029F4D601ED908D0121E007C0BE2DBB321F
:10A2A00019F4F601E1908F0120E068010894C108DB
:10A2B000D108C6016CEC72E143E050E029830E94B2
:10A2C000B1522981009711F572E0E72EF12CE00ED2
:10A2D000F11EC7016FEC72E145E050E00E94B152FF
:10A2E0002981009729F467E0E62EF12CE00EF11E9B
:10A2F000A114B10421F0D5011196FC92EE9220FF39
:10A300000FC130E020E090E88FEF12C1C60164ED8C
:10A3100072E143E050E029830E94B1522981009705
:10A3200031F060E070E0CB01662477240AC0A1140C
:10A33000B10409F4F9C00E5F1F4FF50111830083CA
:10A34000F3C03E2D30533A30A0F52260E22FF0E00A
:10A35000AF014870507022FF07C04115510571F5DB
:10A360000894611C711C2AC04115510519F008940C
:10A37000610871086B017C0152E0CC0CDD1CEE1C05
:10A38000FF1C5A95D1F76C0D7D1D8E1D9F1D660F0C
:10A39000771F881F991F630F711D811D911D6839DB
:10A3A000F9E97F07F9E98F07F9E19F0738F02460A1
:10A3B00005C03E3F39F423FD3FC02860D801ED9031
:10A3C0008D01BFCF353311F03531B1F5F801319141
:10A3D0003D3211F4206102C03B3241F4D8011196A4
:10A3E0003C911197319642E050E002C041E050E0CC
:10A3F00030533A3020F08F01041B150B1DC040E094
:10A4000050E0BCE040385B075CF4DA01AA0FBB1FE8
:10A41000AA0FBB1F4A0F5B1F440F551F430F511D4F
:10A42000319130538F013A3060F324FF03C05095CF
:10A4300041955F4F640E751EC22EDD2421FF08C0BA
:10A44000A114B10429F001501040F50111830083DB
:10A450000E945F4A7B018C01F3E0CF22DD2433E0D0
:10A46000C316D10421F417FB109517F91095C801F4
:10A47000B70120E030E0A9010E94C249882309F415
:10A480004AC077FE09C04BEEC42E42E1D42E709430
:10A4900061947108739404C033E0C32E33E1D32E6A
:10A4A00026E0822E912C90E2A92EB12C0FC0F6014D
:10A4B0002591359145915491C801B7010E94154BE2
:10A4C000E62EF72E082F192F6A187B086A147B04D2
:10A4D00074F7B594A79408948108910881149104A5
:10A4E00029F08CEF9FEFC80ED91EF0CFB701C8013D
:10A4F000282F220F292F221F2F3F39F020E030E094
:10A50000A9010E94C249882331F482E290E090932D
:10A51000B7038093B6033E2D2F2D902F812F08C0B7
:10A5200030E020E090E803C030E020E090EC8FE7DE
:10A53000F901AC016F2F722F852F942F0F90CF91BF
:10A54000DF911F910F91FF90EF90DF90CF90BF9020
:10A55000AF909F908F907F906F9008959927882754
:10A560000895FB01DC014150504088F08D91813409
:10A570001CF08B350CF4805E659161341CF06B35FA
:10A580000CF4605E861B611171F3990B0895881BB2
:10A59000FCCFDC0101C06D9341505040E0F70895BD
:10A5A000629FD001739FF001829FE00DF11D649FB7
:10A5B000E00DF11D929FF00D839FF00D749FF00D43
:10A5C000659FF00D9927729FB00DE11DF91F639FE4
:10A5D000B00DE11DF91FBD01CF0111240895F894BC
:02A5E000FFCFAB
:10A5E2002845787450777229000061747870777208
:10A5F2006F6B005874616C00496E7465726E00571F
:10A6020061746368646F67004E6F726D616C004FB6
:10A612004E004F4646004F6E004F6666004869671F
:10A6220068004C6F770001010000C841AE47E13C71
:10A63200AE47E13CAE47E13C0AD7A33B0AD7A33B76
:10A64200053333234100009041000058416666669D
:10A65200410000A0400000204100004041CDCC4C10
:10A662003F0A00007A455802050001010000FF037D
:10A672008A000400000000000000FF0388000500BB
:10A68200000000001A01011403050001020306077D
:10A692000A0B0E0F020306070A0B0E0F2000BD0362
:02A6A2000000B6
:00000001FF
